:020000040800F2
:10000000002000102D70000831300008851F000806
:100010002D300008293000082530000800000000BD
:100020000000000000000000000000002130000877
:100030001D3000080000000019300008FD240008F1
:10004000957000089570000895700008957000087C
:1000500095700008957000080D4E0008394F000893
:10006000FD4E0008C14E0008854E0008A96C00082E
:10007000996C0008896C0008796C0008696C0008AC
:10008000556C0008416C00089570000895700008D8
:10009000F53000089570000895700008494E00087A
:1000A0001D220008692200089570000891220008AE
:1000B0005D2200084D220008957000089570000828
:1000C00095700008957000089570000895700008FC
:1000D00095700008AD2500089570000831250008CE
:1000E000D14D000895700008AD68000895700008B3
:1000F0002D220008957000083D2200089570000828
:1001000000000000000000000000000095700008E2
:1001100095700008957000089570000895700008AB
:100120002D6C0008196C0008056C0008F16B0008C4
:10013000DD6B000895700008000000000000000062
:100140009570000895700008957000080000000088
:10015000000000000000000000000000000000009F
:100160000000000000000000957000089570000875
:100170009570000800000000000000000000000072
:0801800000000000957000086A
:100188002DE9F04FB54E9DB006F1010906F1020BBD
:10019800741E002554F80B0C88B3B14BCC2707FB11
:1001A800053708E0242838D0AE4B9B7E834200F008
:1001B800D28054F80B0C03685B689847F8B154F880
:1001C8000B0C0368DB68984714F8033C002BE9D054
:1001D800012B26D0022B2AD0032B3BD0042B00F076
:1001E800A980052B43D0062BE3D114F8027C002FFD
:1001F8004ED0012F00F0EC80002304F8033C0135B9
:10020800032D06F1CC0609F1CC090BF1CC0B04F156
:10021800CC04BFD11DB0BDE8F08F012304F8033C26
:10022800C7E74D2812D0002304F8033CC1E7002398
:100238003C2804F8033C00F088803E28B9D101220C
:10024800032304F8022C04F8033CB2E7022304F861
:10025800033CAEE7C028E6D80022042304F8060CC5
:1002680004F8050C04F8072C04F8033CA1E714F87B
:10027800073C14F8062C9A4274D814F8053C8342BB
:10028800D1D114F8027C062304F8033C002FB0D126
:10029800754B14F804AC14F806ECADF82A700FCBC3
:1002A8000DF1100888E80F00631E03EB0E010FFA2A
:1002B8008AF20893BAF1380F4FF001030991ADF8AB
:1002C8002820ADF818208DF82C3000F0EA8354D996
:1002D800BAF1800F00F0FC8300F2A280BAF1520F4D
:1002E80000F0C98440F2DD81BAF1540F00F00084B7
:1002F800BAF16E0F40F076825C4ADFF898A1128856
:10030800DAF808100093FF2A594B5A480490A8BFFE
:10031800FF2281F3100189B240461A7006F066F890
:100328003946404606F062F8DAF8001001F30F018A
:1003380089B245E014F8053C04F8040C584005233C
:1003480004F8050C04F8033C33E7032204F8023CE4
:1003580004F8032C2DE7484A484B49491160494A9B
:10036800DA6026E714F8052CF9184240013304F83E
:10037800052C04F8073C88721BE7BAF1040F00F05B
:10038800CC8340F28B80BAF1200F00F0538440F206
:100398006F81BAF1240F00F04184BAF1280F40F0C0
:1003A80021820093DFF8F0A0314B3748374ABAF87A
:1003B800001004901A60404606F018F8BAF80210C7
:1003C800404606F013F80DF13008009B049A79E0D6
:1003D80014F8042C14F8063C611E0B4408916E2A8C
:1003E8004FF000010A9109930B91ADF8282000F015
:1003F8004A83B62A7FF400AF14F8012C0894042A23
:100408003FF6FAAE01A151F822F000BFA10700089B
:10041800010200087F07000825070008990700085F
:10042800BAF1820F00F0C883C0F04F81BAF1A00F73
:1004380000F08683BAF1FE0F40F0D481144F07F123
:10044800080A37F8021B404605F0D0FFBA45F8D134
:10045800049A012300270DF1300833E0A809002091
:100468009C090020C8130020949200080C1B00204F
:10047800741C0020751C0020FC9F002000ED00E08B
:10048800EFBEADDE0400FA05781C002001060A0163
:10049800141B0020981A0020D41A0020BAF1020F69
:1004A80000F0088100F22F839A4540F09B81C04BF1
:1004B800BF491F70242283F801A08A705346CA1CC2
:1004C8000DF1300854F80B0CADF81A30016805929C
:1004D800D1F820C0B6490491BCF1000F00F09C820D
:1004E800E047BDF91A30059A049954F80B0CA2EBB1
:1004F800010A0022C8F80020C8F804205246FF2A42
:100508004FF0240E4FF04D01A8BFFF2201338DF8A4
:1005180030E08DF8311000F0B4829DF81C30002BCB
:1005280014BF3C213E21BDF818308DF83210BAF1C5
:10053800FE0F8DF833208DF8343040F36F824FEA88
:100548002A238DF8363003238DF835A0009307222F
:10055800414603F093FF009A9DF834309DF833101C
:100568000132022A83EA01030AD0042A9DF83510D1
:1005780008BF9DF8362083EA010304BF5340DBB26D
:10058800BAF1000F8DF80F3057DD5246049954F830
:100598000B0C03F073FFAAF1040189080AF1FF327A
:1005A800013104989DF80F300090062A4FEA81081F
:1005B80040F375824FF0000E8446CDF804B07046C3
:1005C8005CF804BB0EF1010E71458BEA0000F7D808
:1005D800C0F3072141404B40C0F307414B4000990D
:1005E800DDF804B083EA1063C2454144A2EB080277
:1005F800DBB220D00878002A83EA00031BDD4878A4
:10060800012A83EA0003DBB215DD8878022A83EA2F
:10061800000310DDC878032A83EA00030BDD08799C
:10062800042A83EA000306DD4879052A83EA0003E1
:1006380001DD8A7953408DF80F3054F80B0C0122F4
:100648000DF10F0103F01AFF54F80B0C03685B6AF5
:1006580003B19847002304F8033C002F3FF4CFADC3
:1006680054F80B0C05F0FEFB54F80B0CB847C6E524
:10067800BAF1050F40F0B68040460B224D49009371
:1006880005F093FE404608224B4905F08EFE404691
:1006980007224A4905F089FE0DF13008009B049AAB
:1006A80010E7BAF1440F40F09D80049A444F0DF1D1
:1006B800300807E740460422424900930DF130080C
:1006C80005F073FE009B049AFCE63F4A019311680B
:1006D800374B3E48926804904FF6FF7A5145A8BFC1
:1006E80051464FF00A0E21EAE171404683F800E0D6
:1006F80089B2009205F07AFE009A02EB8201490065
:100708005145A8BF514621EAE171404689B205F03A
:100718006DFE0DF13008019B049AD3E6A3EB0B079D
:100728001E2FA8BF1E270DF13008237801933A46E3
:100738006378009359464046CDF820B008F014FD80
:100748001CAAD319224A00214046D2F800A003F877
:10075800401C06F04BFC0099DDF804E0DAF8007064
:100768008AF80BE008448AF80A00434672467F6913
:100778005046B84740E5164B1F683B6838469B68AB
:100788009847144A0123FF2179733B73137033E5AB
:10079800114B01221A702FE501F060FE0F4A104B31
:1007A80000F5742000F51070106000221A7023E51F
:1007B800741C0020009600080C9600081896000883
:1007C800911B0008F8950008D81A0020751C002015
:1007D800200C0020260C0020240C0020300E0020C5
:1007E800250C0020BAF1650F00F01C81BAF1960FB4
:1007F80000F01881AAF1210ABAF1360F00F2078138
:10080800DFE81AF05700050105010501050105019A
:100818000501050144000501050105010501050162
:100828000501050105010501050105010501050190
:10083800050105013700050105010501050105014F
:100848000501050105010501050105010501050170
:100858000501050105010501050105010501050160
:100868000501050105010501A70005019A0005011B
:10087800730014F8013C0A2B00F0C082CDF820B0B8
:1008880001230DF13008049A00271BE614F8013CF7
:1008980008940A2B08A840F0BE8205F07BFDB34FF0
:1008A800388008A805F076FD0DF13008788001231E
:1008B800E9E71CA8AE4F14F8011C2278637840F8C9
:1008C800509D79703A70BB7005F064FD089B3881C3
:1008D800591C1A46089112F8021B797108925B7824
:1008E800BB710DF130080123CDE704F136030DF19A
:1008F800300814F8012C00920893C446274604F1E6
:10090800300A38687968BA68FB68E646AEE80F00CE
:1009180010375745F446F4D13868BB88954ACEF865
:100928000000AEF804301378002BFCD1924B1F78EE
:10093800002F00F01382FEE714F8013C0894FF2B07
:1009480065D18E4B227808961A7001230DF1300874
:1009580099E714F8012C0894032A58D8531E88489C
:100968008849DBB203EB430300EB43030A70587872
:10097800002AEAD00EF1FF33DBB2834247D10022CE
:10098800C1F80220C1F806208A72002B35D02278DF
:100998000896012B8A7030D06278CDF82090022B0F
:1009A800CA702AD0A278CDF820B0032B0A7124D0BF
:1009B800201DE2780890042B4A711ED0601D227910
:1009C8000890052B8A7118D0A01D62790890062B13
:1009D800CA7112D0E01DA2790890072B0A720CD0B8
:1009E800082BE2794A7204F108001CBF04F10902DD
:1009F800237A08901CBF8B720892634B1B78002BDC
:100A0800A3D004F0E1FD0DF1300801233BE74FF0DE
:100A1800FF330DF1300836E75C4968E501230093A0
:100A2800052295E55A4B4046B3F8201105F0DEFC47
:100A3800584BB3F87012404689B205F0D7FC002134
:100A4800404605F0D3FC0021404605F0B8FC049B65
:100A5800514A591C002704911F7011886429A8BFA6
:100A68006421404605F0C2FCBAF1960F00F0688197
:100A78004046394605F0BAFC0DF13008049A0123C6
:100A880020E521214FE508A8089405F083FC08A873
:100A980005F080FC08A805F07DFCFFF7ADBB01461A
:100AA800A8E53E4A394992F801E090780B70117830
:100AB800364A117182F805E005214FF00A0ED77009
:100AC8009071517082F802E00DF130080732F9E4B4
:100AD8003349344A0988901EFF29A8BFFF214FF0E7
:100AE8000A0E02F8011C80F800E00DF13008E9E474
:100AF8002C4A2249901E097802F8011C1221017023
:100B08000DF13008DEE4214802220321427087708B
:100B18000170C21C0DF13008D4E452464046224907
:100B2800009305F042FC3946404605F05FFC049A04
:100B3800009B511C04911370049A0DF13008C1E414
:100B48001A4A00934046116805F039FC184A404695
:100B5800116805F034FC174A4046116805F02FFC6F
:100B68000DF13008009B049AACE400BFD41A0020B1
:100B7800A81A0020270C0020340E0020BC130020E7
:100B8800BC94000890170020501B0020741C002003
:100B9800E40100209C090020481B00208812002046
:100BA8001C1B0020761C0020020C0020ACF7FF1F45
:100BB800B0F7FF1FB4F7FF1FA549A64A08781189A7
:100BC800A54A009302F8010C4046049205F00EFC79
:100BD800A24A04991288DFF8B4A2FF2AA8BFFF220C
:100BE800481C04900A70DAF8082082F3100291B2C7
:100BF800404605F0FBFBDAF8001001F30F0189B25B
:100C0800404605F0F3FB9649049A0978501C049075
:100C18001170009B049A0DF1300853E4914A009337
:100C28004046D2F86C1205F0CAFB0DF13008009B63
:100C3800049A47E48C4ADFF81CA20093D31E9AF862
:100C480001009AF800109AF802E002F8030C5970B3
:100C58004046BAF8081083F802E0049205F0C6FB93
:100C6800049A9AF80510501C04901170049A9AF886
:100C78000610501CCBE77D497D4ADFF814C208787E
:100C8800C2F800C04FF0090E4FF0030C82F805C0FF
:100C98009371D07182F804E002F1080C002800F08A
:100CA800A7800138C0B2DFF8ECE100EB40000EEBA2
:100CB80040004078002800F09B8091F802E082F81C
:100CC80008E001280CF1010240F2B080093ACB7823
:100CD8005372022800F0B5800B799372032802F151
:100CE8000B0300F0A780A3F10B074A79FA720428D6
:100CF80003F1010200F098808A793A73052803F11C
:100D0800020200F09180CA797A73062803F103027F
:100D180000F08A800A7ABA73072803F1040200F007
:100D280083804A7AFA73082803F105027CD08A7A0C
:100D38003A740DF130089A1D00270123FFF7C2BB52
:100D4800049A0123D11804911370049AD1180491BC
:100D58001770049A0DF13008FFF7B4BB454B1868BB
:100D6800454B4FF0010A83F800A004F001F8434A0C
:100D7800384682F800A004F0B5FB384604F0B2FB10
:100D8800092004F0AFFB009804F0ACFBC246AAEBC4
:100D98000807FFB20A2004F0A5FB384604F0A2FBBE
:100DA8001AF8017B0B2004F09DFB384604F09AFBEF
:100DB800334B186803F0D3FF0DF166035345E6D1B2
:100DC800082004F08FFBA02004F08CFBA02004F086
:100DD80089FB002004F086FB10F02000F6D1254B9B
:100DE8000746186803F0C9FF234B1F7001234AE523
:100DF800624607460DF13008FFF764BB214B2278A5
:100E08001A706178A27859709A70CDF820B00123D1
:100E18000DF1300837E505F0BDFA08A805F0BAFA73
:100E28000DF1300801232EE5012300270DF13008CC
:100E3800FFF748BB1A46002701230DF13008FFF7DA
:100E480041BB114A012300270DF13008FFF73ABBD7
:100E5800941A0020A81A0020751C00200C1B0020E2
:100E68006C1C00209C090020771C00209017002093
:100E7800741C0020B4130020340E00203E0E002005
:100E8800A0160020881200207E1C0020981A00203E
:100E980003010602BC94000808B51F4B002832D095
:100EA8001E481A6800210180137813F07F0316D0BA
:100EB800012B27D0022B24D1527902F00F039B007B
:100EC80003F1804303F5B84312061B681FD403F4EB
:100ED8004053B3F5805F0ED1012303700BE0527AC3
:100EE800930654BF0378022351064CBF43F0010315
:100EF80023F0010303700A4B1B681B6998470748D6
:100F080008BD084608BD1B6802221A8208BD03F006
:100F18003003102BEFD1DFE7EC1500201C0C00206C
:100F28001016002008B538B1064B1B689B68984717
:100F3800054B18680C3008BD034B1B6801221A8248
:100F480008BD00BF10160020EC15002008B538B108
:100F5800064B1B681B689847054B18680A3008BD84
:100F6800034B1B6801221A8208BD00BF101600201F
:100F7800EC15002010B5094C60680368DB699847D8
:100F880050B9237A0BB9637A33B160680368DB68B8
:100F9800984700232372A37210BD00BF1C0C0020C9
:100FA8004FF0FF30704700BF0020704700207047A7
:100FB800014BD87A704700BF1C0C002010B40548BC
:100FC8001E2404FB0211014400200B735DF8044B3E
:100FD800704700BF1C0C0020F0B41C7894B11E2090
:100FE8000A4F10FB021200200D181D2D07EB0005FB
:100FF80000F10106D8BFAD18F0B2D8BF2C731C5C45
:10100800002CF1D10020F0BC704700BF1C0C002060
:10101800014B1888704700BF00000020002070476F
:10102800002302220271037043708370C3707047FB
:10103800024B1A889B78028083707047A49200083C
:1010480038B50F4C637AA3B9D4F81432C01A002803
:101058000FDD60680B4B056816210C228172C27285
:10106800012161726D690821A847606803685B6A9D
:101078009847A07A10B9207A00B9607A38BD00BFC5
:101088001C0C00202496000838B50B4C94F8183234
:1010980005460BB905F070FC084B94F81D129A78B8
:1010A80094F81C3212F0400F14BF10220D220A448B
:1010B8001E332A726B7238BD1C0C00200000002001
:1010C80070B51F4C94F81E32ABBB94F8213203F074
:1010D800F7031C4E84F82132306803F049FE94F877
:1010E8002152042004F0FEF9284604F0FBF9306888
:1010F80003F043FE94F8205294F81F323068C5F18B
:10110800030545EA830503F033FEEDB21024E0B28F
:1011180004F0E8F90134284604F0E4F9202CF6D16B
:10112800306803F02AFE21464FF4F072064808F0B2
:1011380040F8002070BD94F8213243F00803C8E756
:101148001C0C0020B4130020280C00200F4B104A60
:101158001B689BB223F0070303EBC00002443E293F
:101168004FEA42020AD94B09C80604BF03F1FF330C
:101178009BB29B0243F40043136070474B08C907B6
:1011880048BF01339B021360704700BF505C0040AA
:1011980006300020054B064A1B689BB223F0070364
:1011A80003EBC0000244520011607047505C0040DD
:1011B8000230002000230360436083608381036161
:1011C80043618361C361036243628362704700BF06
:1011D800F0B48B680F6A0E694D698A69CC693B4324
:1011E80033432B434E6A8D6A8F8913430268234326
:1011F800334322F4FF422B4322F070020C6813435E
:101208004A68036047608460C260F0BC704700BFF2
:1012180002683B494FF6FE731A4088424FF00003BC
:101228000260036043608360C36027D0354B9842F7
:101238002AD0354B98422DD0344B984230D0344B7D
:10124800984239D0334B98423CD0334B98420FD018
:10125800324B98423CD0324B98423FD0314B984267
:1012680042D0314B984245D0304B98421ED07047FF
:101278002F4A536843F07063536070472C4A536891
:1012880043F00F0353607047294A536843F0F00353
:1012980053607047264A536843F47063536070473D
:1012A800234A536843F4704353607047214A536894
:1012B80043F470235360DAE71D4A536843F47023FC
:1012C800536070471A4A536843F470035360704779
:1012D800184A536843F00F0353607047154A536820
:1012E80043F0F00353607047124A536843F4706345
:1012F800536070470F4A536843F470435360704714
:10130800080002401C000240300002404400024035
:10131800580002406C00024080000240080402406D
:101328001C040240300402404404024058040240B5
:1013380000000240000402402DE9F04F764C94F87A
:1013480018328FB013B994F822521DB100200FB093
:10135800BDE8F08F714F724E3868DFF8E0810123E5
:1013680084F8183203F004FD802004F0BBF8284606
:1013780004F0B8F80546386803F0FFFCB378D8F8ED
:101388000020AB423DD005F05BFB0022B4F82C32C4
:10139800B6F800C04FF0050A16464FF006094FF0A0
:1013A8000708E01803F1010E90F83012057BA942F6
:1013B80006F1050113D004EB010BA11980F8305296
:1013C800180A81F810A481F8129481F8133481F86E
:1013D800148481F81104013206368BF810541FFA70
:1013E8008EF3634502F101022CD2632AD9DDA4F8F9
:1013F8002C325EBB0023002084F818320FB0BDE801
:10140800F08F484B1D78002DBFD1D4F82432D31A61
:10141800B3F57A7FB9D93868019203F0A9FCA02006
:1014280004F060F8284604F05DF88146386803F057
:10143800A4FC19F0040F019A50D0C4F82852C4F83B
:101448002422A2E70023A4F82C32D2E71FFA86F957
:10145800E37A03F0FF05002BFAD1DFF8E480324E7F
:101468004046FFF7D5FE3046FFF7D2FE03A8FFF748
:10147800A1FE2E4A2E4B099503A930460A950795D9
:101488000B950C950595089503920493ADF8189063
:10149800FFF79EFE3368274D43F0010333601022A7
:1014A800802303A94046059208930495FFF790FE10
:1014B800D8F80030386843F00103C8F800303368C2
:1014C80043F00203336003F053FC01231A4AE3722A
:1014D80093889BB243F0030393808BE709F00503DD
:1014E800012B11D0002BAAD1B3785B06A7D5D4F86D
:1014F8002812D8F8003059B15B1A642B9FD9019291
:1015080005F09EFA019A9AE7B3785906EFD596E75F
:10151800C4F8283293E700BF1C0C0020B413002045
:1015280000000020B8130020440002400C3800409E
:10153800040000202C100020003800404017002034
:1015480058000240084BDA68D1070BD4DA68D20693
:1015580001D502207047DB6813F0040F14BF032085
:10156800042070470120704700200240B64B59689C
:1015780001F00C0104292DE9F04100F08D810829C2
:1015880000F07681B14A026001B10021DFF8B8E2CB
:10159800AF4CDEF80430C3F3031323441E7AF6B2CB
:1015A80022FA06F34360DEF80450C5F30225254409
:1015B8002F7A23FA07F78760DEF80450C5F3C225AF
:1015C80025442D7AEDB2EB40C360DEF82CC04FEA1B
:1015D8001C1C0CF00F0E04EB4E0E1CF0100FBEF886
:1015E80018E01FFA8EFE03D0BEF1000F40F0A8806D
:1015F8009646DFF854C2C0F810E0DCF82CE04FEA59
:101608005E2E0EF00F0C04EB4C041EF0100F248B12
:10161800A4B202D0002C40F090801446DFF828E2F3
:101628004461DEF830C0894C1CF0100F0CBFA44692
:101638009446C0F818C0DEF830C01CF0200F0CBF6C
:10164800A4469446C0F81CC0DEF830C01CF0400F19
:1016580018BF14460462DEF83040E40502D5914212
:1016680000F0CC80784C4362D4F830E01EF4805F00
:1016780057D0914200F02B818362246BA40540F17E
:10168800CF80714CC362D4F830E04364246B2405E6
:1016980040F1E0806C49096B83646B490C6BA507CA
:1016A80052D00B6B03F00303012B00F007810B6B87
:1016B80003F00303022B00F036810B6B03F00303E6
:1016C800032B40D0604B196B11F4403F42D1476364
:1016D8005D4B196B11F4402F57D187635A4B196B27
:1016E80011F4401F6CD1C763574B196B11F4400FAD
:1016F80000F08180196B01F44001B1F5800F00F012
:10170800E3801A6B02F44002B2F5000F00F0138177
:101718001B6B03F44003B3F5400F00F0C980BDE82C
:10172800F0818362246BA4057AD59142A9D1AE4297
:10173800A7D14FEA410C6446D5E0B1FBF4F46DE75C
:10174800B1FBFEFE55E7414B03633F4B196B11F4A8
:10175800403FBCD0196B01F44031B1F5803F00F037
:10176800AF80196B01F44031B1F5003F00F0DF8024
:101778001B6B03F44033B3F5403F04BF334B436363
:10178800314B196B11F4402FA7D0196B01F440218C
:10179800B1F5802F00F09680196B01F44021B1F566
:1017A800002F00F0B8801B6B03F44023B3F5402FE3
:1017B80004BF264B8363244B196B11F4401F92D04E
:1017C800196B01F44011B1F5801F75D0196B01F444
:1017D8004011B1F5001F00F0A2801B6B03F4401309
:1017E800B3F5401F04BF194BC363174B196B11F4B2
:1017F800400F7FF47FAF0764BDE8F081AE427FF40D
:1018080031AF4FEA410CC0F824C0DEF8308018F43C
:10181800805F64465FD18362DEF83040A4058AD4D5
:10182800094CC362246B640501D591423CD0064C37
:101838004364246B24050DD591427FF42BAFAE424F
:101848007FF428AF54005EE00010024000127A00D6
:10185800000000203A4C8364246BA4047FF51CAF7D
:1018680091427FF419AFAE427FF416AF540050E0B6
:1018780059685A68C1F38341D50301F102010FD5B4
:10188800DB6A304A03F00F030133B2FBF3F301FBC9
:1018980003F101600A4679E62A4A0260002175E6EA
:1018A800294B03FB01F1F4E7AE42C0D14C0022E022
:1018B800244B0364BDE8F081C26315E7026301E7C6
:1018C800426305E7826309E70264BDE8F081AE423E
:1018D8007FF4D2AE4C00DFF868E08462DEF830E0D6
:1018E8001EF4007F9CD0DFF858E0C462DEF830E0D8
:1018F8001EF4806F9BD0DFF848E04464DEF830E0E7
:101908001EF4006FA6D00E498464096B8D047FF520
:10191800C3AEC464C1E64FF400438363DEE64FF40C
:101928000043C363E0E64FF400430363CAE64FF4A1
:1019380000434363CCE64FF400430364BDE8F08101
:101948000010024000127A0000093D00F0B504467C
:101958000068D1F808E04B68CF680E6920F00100F4
:101968000D4649692060626822F4405242EA0E023C
:10197800626022683B4322F4B05222F00C023343E7
:1019880013432360A36823F440730B4395B0A3600B
:101998006846FFF7EBFD174B9C4224D0164B9C4240
:1019A80023D0164B9C4222D0154B9C420CBF0F9A59
:1019B800109A23682968180448BF5200B2FBF1F353
:1019C80001FB1322B2EB510F226828BF0133120426
:1019D80005D54FF6F0721A40C3F3420313439BB286
:1019E800A38115B0F0BD0C9AE3E70D9AE1E70E9AD2
:1019F800DFE700BF003801400044004000480040D5
:101A0800004C004000222DE9F04313460F680126E0
:101A18004FF0030E04E00133102B02F1020224D030
:101A280006FA03F434EA0705F5D10D7905F1FF3C10
:101A3800BCF1010F0EFA02FC19D96FEA0C0C04680C
:101A480004EA0C0404600468954025430560C568F1
:101A5800CC790EFA02FC944025EA0C0501332C439C
:101A6800102BC46002F10202DAD1BDE8F083D0F88D
:101A780008800EFA02FC6FEA0C0C08EA0C08C0F8A1
:101A8800088091F80580D0F8089008FA02F848EA2A
:101A98000908C0F80880B0F804801FFA88F828EA16
:101AA800040484808C79B0F804809C4044EA0804DB
:101AB800A4B28480C3E700BF2DE9F0430368244F34
:101AC8009B687860044689B098474FF00108FF2367
:101AD800637384F80C80A024FF2C19D05FFA88F671
:101AE800234600257868E9B201F1040E026880F8FF
:101AF8000AE0C6720331D2F8189001340135C9B230
:101B08003246C847E4B2182D234602D0FF2CE9D14B
:101B1800FF2408F10108B8F1050FDDD168460D4A28
:101B28000D4900F07DFD6B4606221421786803F00C
:101B38003FFA06220D21094B786803F039FA7868D4
:101B480003685B6A984701233B7209B0BDE8F083DC
:101B58001C0C0020349600083C96000840960008AB
:101B680038B5084D00242B59CC3418461BB11B68D6
:101B78005B68984720B9B4F5197FF4D1002038BDC7
:101B8800012038BD9C090020014B024ADA60FEE7BB
:101B980000ED00E00400FA05012312211322417030
:101BA80042710370037170472DE9F0410B78057B92
:101BB800DB43DFB200F1130200F11D0302F8015FFD
:101BC8009342FBD1DFF890E000F12701002203F8EF
:101BD800012F9942FBD114210524002647FA04F36A
:101BE80003F00103002B1E4414BF4FF019084FF0F7
:101BF8000A0814F0010FF6B214BFAC464FF0000CFF
:101C08000023CA1810FA82F20133434582F814C03F
:101C1800F7D15A1E92B20132013C8B18621C9BB25A
:101C280001D01946DAE716F0010F14BF19240A2467
:101C38000022991810FA81F10132A2420D75F8D1EB
:101C480013449BB25A1C0344002192B21975AEF892
:101C580000200261BDE8F081941200202DE9F04FC8
:101C6800DFF890A0BAF802300B3383B01FFA83F97B
:101C780001F1060B4FF001084FF0000C002711F896
:101C880001EB3E464C460122A4F10B039BB20191A5
:101C980005E001339BB2017B29759C4208D0C51829
:101CA800002AF6D1C51801339BB29C422A75F6D199
:101CB80003190136092F019983F814C0F6B20CD024
:101CC800092E15D008FA07F313EA0E0F14BF0122E4
:101CD80000220C34A4B20137D6E709F17809594536
:101CE8001FFA89F9CAD1AAF802C003B0BDE8F08F7B
:101CF8000022EEE7941200202DE9F047DFF85C801F
:101D0800B8F8043004331FFA83FC01F109094FF0D5
:101D1800010E11F8017B64460026231F0EFA06F215
:101D28009BB23A40C2B1B0F80CA0C51801339BB2BF
:101D38009C4285F814A0F5D101360434082EA4B2CB
:101D4800EBD10CF1200C49451FFA8CFCE1D10023A2
:101D5800A8F80430BDE8F0879246E6E79412002020
:101D680010B40268047B11680223A340194209D009
:101D78000649406800240C7001684FF6FE74214043
:101D8800016053605DF8044B704700BF8C1700205A
:101D9800436A8269D154436A0169426B01338B42B9
:101DA80028BF00234362002A2FD0EFF3118150236C
:101DB80083F31288436B1A68D2072CD470B45E6818
:101DC8006EB9456A826A954217D084691444DC600A
:101DD8000ED9AA1A5A608562002280F850201A6823
:101DE80042F00102C9B21A6081F3118870BC7047D1
:101DF8000469A21A5A608662EEE7012380F850301F
:101E0800C9B281F3118870BC7047C26C136843F083
:101E1800800313607047C9B281F31188704700BF0F
:101E2800026B10B462B1036CC2684469D11A013BF9
:101E3800615C5DF8044B08BF13460364C8B2704781
:101E4800016A4369C4685B5C0131A14228BF11463D
:101E580001625DF8044BD8B2704700BF436B13B101
:101E680090F850007047836A406A181AB0FA80F0F8
:101E780040097047416A836A99420AD3CB1A416B79
:101E8800026961B14968501E0B4483420AD2C01AE4
:101E9800704702691144CB1A416B0029F2D1501ED8
:101EA800C01A704700207047036B43B1026C5B682F
:101EB80093422FBF981AC0689B1AC0187047C2690E
:101EC800036A9A422FBFD01AC0688018C01A704798
:101ED8002DE9F0470569C3681D4028D00F4606461E
:101EE8004FF000484FF00009B5FA85F328FA03F2DD
:101EF800D2431B3B32611540042B16D8DFE803F0B0
:101F08003129211903007B6A002B32D003F1FF3AF3
:101F18001FFA8AFAC7F824903C6A34B1236820462D
:101F2800514698476468002CF8D1002DDCD1BDE8F3
:101F3800F0873868716B036889B29847002DD3D150
:101F4800F5E77868B16B036889B29847002DCBD163
:101F5800EDE7B868F16B036889B29847002DC3D1E3
:101F6800E5E7F868316C036889B29847002DBBD162
:101F7800DDE7F36A1FFA83FACEE700BF184C08B50D
:101F88000121022002F008FFA37903F00903092BBD
:101F980008D00021012002F0FFFE0021084602F0CF
:101FA800FBFEFEE70F4A104B11681A680B68A06821
:101FB8004FF6FE752B400B60138823F001031B04BA
:101FC8001B0C138018B1292200238271C3710222CD
:101FD8004E2102F037FBA06802F0CAFED9E700BF25
:101FE800941200205C1B0020601B00202DE9F04F9C
:101FF800F022002183B07848784CDFF80492784DBD
:10200800784E794FDFF8FC8107F0D3F877487849A4
:10201800DFF8F4E1DFF8F4C100221359834200F03D
:10202800C180B3F1804F00F0BF80AB4200F0C880A0
:10203800B34200F0C780BB4200F0C680734500F091
:10204800C580634500F0C480434500F0C380DFF8D5
:10205800C0A153457ED00AF5806A534508BF0923BD
:1020680079D01432F02AD8D15C4C624D624E604F60
:1020780004F1F00802E01434A04568D0A379002BDD
:10208800F9D023794FEA131909F1FF39B9F1050F8E
:1020980003F00F03EFD835F8190040FA03F2D2071E
:1020A800E9D54FF0010A0AFA03F3013B184004F09E
:1020B800A5FF16F809305149184411EBC002DAD0CF
:1020C80051F830004E4B217A00F1384E03EB9E2335
:1020D80093F8503003F01F0E5B09022B0AFA0EFA30
:1020E80069D0032B62D0012B03D17B694AEA030331
:1020F8007B6193880093B3FA83F3C3F11F039BB208
:10210800DA0800EB820203F00703D2F820E09B0014
:102118004FF00F0C0CFA03FC2EEA0C0EC2F820E06C
:10212800D2F820E001FA03F343EA0E03136269468A
:102138000023022214348DF804208DF805308DF820
:1021480006308DF80730FFF75DFCA04596D103B047
:10215800BDE8F08F082309EBC3034FF0010B93F898
:1021680004A00AF01F034FEA5A1ABAF1020F0BFA39
:1021780003F30BD0BAF1030F0ED0DA457FF471AF39
:10218800D1F814A043EA0A034B616AE7D1F818A012
:1021980043EA0A038B6164E7D1F81CA043EA0A0307
:1021A800CB615EE70023D6E70123D4E7FB694AEA5F
:1021B8000303FB619DE7BB694AEA0303BB6198E738
:1021C8000223C8E70323C6E70423C4E70523C2E7BD
:1021D8000623C0E70723BEE7A0120020CC9300081F
:1021E800000400400008004000100040002C01409E
:1021F800001002406093000858930008441400201F
:10220800A89200080040014000140040003401403A
:1022180000440140014902485AE600BF401300202B
:10222800004001400149024852E600BF181300204F
:1022380000340140014902484AE600BF1813002053
:10224800003401400149024842E600BFF012002074
:102258000004004001494FF0804039E6C8120020D0
:1022680010B5064C064804F10C01FFF731FE04F1E5
:10227800D4010448BDE810402AE600BF94120020AB
:10228800002C0140004401400149024820E600BFFB
:10229800A0120020002C01401F4B98422CD0B0F116
:1022A800804F2BD0A3F59433984229D003F580634F
:1022B800984227D003F50063984225D003F5806340
:1022C800984223D003F59033984221D003F5406318
:1022D80098421FD003F58063984207D003F58063C6
:1022E800984208BF092202D00020704708220B4BF1
:1022F80003EBC203187970470022F8E70122F6E7DA
:102308000222F4E70322F2E70422F0E70522EEE7CF
:102318000622ECE70722EAE7002C0140A892000811
:102328002DE9F04FDFF830C1474A4849484E494D3A
:102338008046102718F1FF38C0F08480DCF804309C
:10234800C3F30803002B5CD1EFF31183002B58D1A2
:102358000B68946800BF08688342F9D1D6F80090EA
:102368004FF47A7000FB09FEAEEB040EBEFBF9FEDB
:1023780000FB03EEDCF80430C3F308034FF47A746F
:102388000120FBB9EFF31183E3B90B68D2F808A079
:1023980000BFD1F800904B45F7D1D6F800B004FB48
:1023A8000BF9A9EB0A09B9FBFBF904FB0393A3EBAF
:1023B8000E03B3F57A7FBDD2DCF80430C3F308030B
:1023C800002BDFD0EFF3118A87F31288D2F808B018
:1023D8001368DB0344BF2860D2F808B00B68D5F84F
:1023E80000905FFA8AFA8AF31188D6F800A0994417
:1023F80004FB0AF3A3EB0B03B3FBFAF304FB093367
:10240800D5E7EFF3118487F31288D2F808901368A0
:10241800D80303D501232B60D2F808900B682868ED
:10242800E4B284F31188D6F800A04FF47A7400EB74
:10243800030E04FB0AF3A3EB0903B3FBFAF304FB53
:102448000E3E97E7BDE8F08F10E000E0401700204F
:10245800441700203C17002000ED00E0204B5B688B
:10246800C3F3080330B4BBB9EFF31183A3B91D4B11
:102478001D4C1868A16800BF1A689042F9D11B4B1F
:102488001C684FF47A7202FB04F3591AB1FBF4F199
:1024980030BC02FB00107047EFF31182102383F366
:1024A800128811498C680B6813F4803F104B02D0D6
:1024B800012018608C680B49D2B20D68186882F345
:1024C80011880A4B19684FF47A72284402FB01F309
:1024D8001B1B30BCB3FBF1F302FB0030704700BF9D
:1024E80000ED00E04017002010E000E04417002055
:1024F8003C17002030B4EFF31183102282F31288C6
:102508000649074C0A680748013200250A60256019
:10251800DBB2026883F3118830BC70474017002093
:102528003C17002010E000E01D4B70B59C68E36C80
:10253800226BDD69C2B1636B2BB12B0702D5E36C4B
:1025480008221A6270BD2A06F7D5A26A616A8A4211
:102558001FD0511CA069A162825C2069E66C81428F
:102568003285EAD3A362E8E7A906E4D5E26A1AB19C
:10257800988C80B29047DEE7E1699B8C6069DBB29A
:102588004E1CE6614354E169E368994228BFE26161
:10259800D1E7E26C136823F080031360CDE700BF36
:1025A800481700201D4B70B51C68E36C226BDD6971
:1025B800C2B1636B2BB12B0702D5E36C08221A62F8
:1025C80070BD2A06F7D5A26A616A8A421FD0511CDB
:1025D800A069A162825C2069E66C81423285EAD3F7
:1025E800A362E8E7A906E4D5E26A1AB1988C80B23A
:1025F8009047DEE7E1699B8C6069DBB24E1CE661BF
:102608004354E169E368994228BFE261D1E7E26C8B
:10261800136823F080031360CDE700BF481700203C
:102628000EB42DE9F04189B010AD684B019000243B
:102638000295039326465622019B591C01910134A9
:102648001A70039B5A1C03921A78002A3ED0252A36
:10265800F2D19A1C049603925878302858D0002753
:10266800A0F13003DBB2092B39D96C283DD064289E
:1026780000F096800FD8252847D06CD9582878D0F4
:102688006328DED1019B2A78591C01911A70013404
:102698000435039BD6E7732853D05FD9752865D1D5
:1026A8000DF114082868434600220A21043503F076
:1026B80039FE43463A46049901A802F0BFFF039B3E
:1026C8005A1C03921A780444002AC0D1019B0022A4
:1026D80020461A7009B0BDE8F04103B0704704AA5B
:1026E80003A902F0E7FF6C28C1D1039B1A46013306
:1026F80003931278642A5BD00FD8252A05D05FD9B6
:10270800582A11D0632ABDD09CE7019B252294E763
:10271800DA1C039298780127A2E7732A11D052D9BC
:10272800752A33D0782A8DD1A2F158014A420DF189
:1027380014084A41286843461021043503F0F2FD85
:10274800B7E72B680499002201A802F077FF043547
:102758000444039B76E70028B8D072E76E287FF41C
:1027680070AF039B2A68043514606BE778287FF400
:1027780068AFA0F158035A420DF114085A4128686D
:102788004346102103F0CEFD043592E70DF11408FD
:102798002868434600220A21043503F0C3FD88E770
:1027A8000DF1140828684146043503F08DFD80E7D3
:1027B8000DF1140828684146043503F085FD78E7D3
:1027C800002A83D03EE76E2ACCD03BE73D9600082E
:1027D80070B5414C414B23602046FEF771FC002543
:1027E8000122FF23222022736373A57301F066FE82
:1027F800206110B12523C5718371492102F0F3F8D6
:10280800206902F0B5FA6420FFF78AFD206902F01A
:10281800B4FA2C2001F052FE606118B11D22002389
:102828008271C3712E4D0D2102F0DDF8606902F04E
:10283800A4FA2B8823F040031B041B0C2B802B8845
:102848009BB223F0380343F010032B802B889BB2F4
:1028580043F040032B800A2002F044FE402002F09F
:1028680041FE8A2002F03EFEFF2002F03BFE2B884C
:10287800606923F040031B041B0C2B802B889BB240
:1028880023F0380343F008032B802B889BB243F0D6
:1028980040032B8002F06CFA002002F023FE022095
:1028A80002F020FE606902F068FA667FA57F237F48
:1028B8000C492376C0220023C6F12006C5F1100575
:1028C8000320E67784F8205004F060F90248FEF708
:1028D800DBFB014870BD00BFA01300200093000877
:1028E80000380040BD6800081C4A92F82430022BCA
:1028F80030D802EBC3011846098D0133C907DBB292
:1029080022D4032B26D002EBC30110B40C8D023065
:10291800E407C1B218460BD4022902D1138FDB0792
:102928000FD4032382F8243000205DF8044B70474D
:102938000B460B4982F8243001EBC0005DF8044BCC
:10294800704708460323F4E7054982F8243001EB71
:10295800C000704782F8243000207047A013002080
:10296800C81300202DE9F043734E96F99230834244
:102978008DB00DD096F99A30834200F0AA8196F96D
:10298800A230834200F0BE8100200DB0BDE8F08384
:102998000027FF00F319B3F89040002CF4D1022867
:1029A800884607D0142800F0C98018B120460DB019
:1029B800BDE8F083C5B22846414602F0DDFC044676
:1029C8000028F3D0C06C00230322A371627102684F
:1029D800236222F0010201210DF10409E361A362DF
:1029E8006362E36284F85010C4F8088049460260C4
:1029F8000C2202930393049306930592CDF8048066
:102A0800FEF7A4FF6079E36CA17900F00202002AC6
:102A180015BF4FF440324FF480324FF4003E4FF070
:102A2800000E10F0010F586808BF724611F0010F30
:102A380014BF024320EA02025A609A6809074CBF91
:102A480042F0080222F008029A601A68216B42F0EC
:102A580001021A60002900F05C814846FEF7AAFBD3
:102A6800A36CE2686169206B01934FF480530A9369
:102A7800002302910B9380210593079308930393F6
:102A88002023ADF8102009930691FEF7C1FB4946B3
:102A9800206BFEF79DFB226BE36C116841F001018E
:102AA8001160996841F040019960526892B22264BD
:102AB800626B002A00F028814846FEF77BFB626CB7
:102AC800236901924FF480524FF00008606B0A921C
:102AD800ADF810308022102306920393CDF82C8095
:102AE800CDF81480CDF81C80CDF82080CDF8248056
:102AF800FEF78EFB4946606BFEF76AFB626BE36C80
:102B0800116841F002011160C2F80480C2F8048023
:102B18009A6842F080029A601A6842F001022046E0
:102B28001A603E4401230571C6F88C00A6F890305F
:102B38000DB0BDE8F08300BFA0130020784D7948A0
:102B4800AB6943F00103AB61112101F04CFF7548FB
:102B580002F00EF902F04EFB724802F00EF96B69B2
:102B68000DF1040943F400336B6103220223494643
:102B78004FF4C0554FF090408DF80A408DF80B4047
:102B880001958DF809208DF80830FEF73BFF4FF0CE
:102B9800904396F84822586ADFF8BCE1624C634DCE
:102BA800634920F470405862586A40F460405862A3
:102BB800586A20F470205862586A40F460205862BD
:102BC8004FF48023CEF8003023685A4823F480233A
:102BD80023602C6802F1804324F480222A6003F5E4
:102BE8008233012208244FF0120EC6F844E286F818
:102BF800494286F84A221C6844F480241C60D6F8AE
:102C0800443223F01F0503F01F036C5802FA03F344
:102C180024EA03036B50D6F8443223F01F0503F06F
:102C28001F032C5802FA03F324EA03032B5096F8E7
:102C38004932102B4FD0D6F8441203F1804321F0CB
:102C48001F0003F5823301F01F01C4588A40224354
:102C5800C250394A3249394BC6F86C3200241460E4
:102C6800CA693748C6F84C0242F40002CA614FF0FC
:102C7800020803F13002C6F870221B6886F85882F1
:102C88009847304B304ADA600125142348468DF8BE
:102C980004308DF805808DF806408DF8075002F055
:102CA8004DFB9DF807308DF805502A228DF8064017
:102CB8008DF804204BB9254B4FF48062C3F884206B
:102CC800234B7364142523482BE7484602F036FB50
:102CD800F6E701275DE6D6F8443223F01F0403F037
:102CE8001F03655802FA03F32B436350D6F84432A6
:102CF80023F01F0103F01F030C5802FA03F32343C8
:102D08000B50A6E7022744E61A6842F080021A60D0
:102D180002E720221A621A6842F020021A60C7E607
:102D280000100240A41400200004014004040140E3
:102D3800080401400C040140D80042423800002039
:102D4800F015002000ED00E00005FA0500E100E0C4
:102D58002C930008E4130020140401400F4B1A8D33
:102D6800D1074FF000000AD41A8ED2070FD4188F5B
:102D780010F001000ED1032283F824207047024688
:102D88000121074883F8241000EBC2007047022194
:102D98000122F6E703210222F3E700BFA013002077
:102DA800C813002030B40D4A002314250224032040
:102DB800C2F89030C2F89830C2F8A030C2F8943007
:102DC800C2F89C30C2F88C3082F89A3082F892505F
:102DD80082F8A24082F8740230BC7047A013002029
:102DE8004348444A018D4B0830B403F077338D08CB
:102DF800CB1A05F03335CC0804F011345B1B1B1BD0
:102E080003EB231303F00F3382FB03421A44D2115E
:102E1800C2EB02229A1A012A01F0010405DD022AF6
:102E280063D101F0810181295FD1058E6908EA0724
:102E380001F077314FEA9502A5EB010102F0333238
:102E48004FEAD503A1EB020203F01133A2EB03030F
:102E580003EB2313274A03F00F3382FB03121A44B0
:102E68004FEAE212C2EB022248BF0134A3EB02028E
:102E780048BFE4B2012A05DD022A36D105F08105F2
:102E8800812D32D1058F690801F07731AA08EB0747
:102E9800A5EB010102F033324FEAD503A1EB0202A0
:102EA80003F01133A2EB030303EB2313114A03F0DE
:102EB8000F3382FB03121A444FEAE212C2EB0222DA
:102EC80048BF0134A3EB020248BFE4B2012A05DD82
:102ED800022A0AD105F08105812D06D1601E02283B
:102EE8008CBF0020012030BC70470020FBE700BFEA
:102EF800A013002081808080704700BF2DE9F04139
:102F0800304E37683A8A2AB93D7A042D43D0BC8AB4
:102F1800042504E0BC8AA2428CBF02250425944201
:102F280028BF14461FFA84F8BB6940469847264BC9
:102F38001B689BB223F0070303F1005303F54053CA
:102F48005B00621C1C68A4B204F1005404F54054F0
:102F580052104FEA440418BF002306D030F8021B71
:102F680024F8231001339342F8D141460020FEF79C
:102F780011F97B8A3A8A1549A2EB08029844302055
:102F88004FF440533A82A7F81280376848808B8004
:102F98003D72BDE8F0810D4B1978012905D0072550
:102FA80010223D725A80BDE8F08107480849006840
:102FB8001A7080B220F007000144490030200A60EE
:102FC8005880E5E7EC150020505C004038160020DA
:102FD8000230002008B50B4B002093F82C10FEF7A8
:102FE800B5F8094B1B68187A082805D1074B4FF428
:102FF8008051102299805A80A0F10900B0FA80F01F
:10300800400908BD38000020EC15002038160020C3
:10301800704700BF704700BF704700BFFEE700BFA2
:10302800FEE700BFFEE700BF704700BF202938B5A4
:1030380003D80D4621BB284638BD20252946102334
:10304800114A30F8024B22F8044C013B02F1040209
:10305800F7D10120FEF79EF80C490D4A0B682B4466
:103068000B60136823F4E04323F040039BB283F022
:10307800300343F4004343F080031360284638BD0F
:103088004B1C5B1089B2DBE78461004054160020BA
:10309800045C0040B2B170B4541EE4B201340023A1
:1030A80064001E46020F092A02F1300586BF373236
:1030B800CA54CD54CA1802339C424FEA00105670C5
:1030C800F0D170BC704700BF064B9B7A23B9064B02
:1030D80001221A6003F0ECBD034B05221A6003F0CD
:1030E800E7BD00BFF015002050160020A1490B686D
:1030F8002DE9F043A04CA14D9BB2E380E2882B88D8
:103108001A40970583B006D54FF6FF520A60227A17
:103118000132D2B22272E2881A40160427D4E28819
:1031280002F48062134219D1E28802F480521342F9
:1031380002D103B0BDE8F0838E4A00234EF6FF713A
:1031480011602373237B052B00F27781DFE813F0EE
:10315800F600E600E100D600CB00B700854A884BB0
:103168004FF6FF315B68116098472B88DCE7002336
:10317800DFF80082834E844FADF80230D8F8002083
:1031880090B213044BF6BF7E48F28001E08040F114
:10319800DC80E38803F00F039A0002F1804202F515
:1031A800B8426372002B63D13B689BB2A380A388AB
:1031B80003F030036380A38803F44053A3803B6883
:1031C80003EA0E0383F4005383F020030B433B60B0
:1031D800E388D80640F1BB803B689BB2ADF802306B
:1031E800BDF802301A0500F1D580BDF80230190487
:1031F800C4D53B68654E40F68F721340D6F8008000
:103208003B6098F80830022B0AD0042B08D0032B17
:1032180000F0F281052B00F0EF81072B00F06382AC
:10322800082388F80830FFF7D5FE574B1B68A2889B
:103238004BF6BF71D204A28803EA010348BF83F4A6
:1032480080539704628848BF83F40053D606628887
:1032580048BF83F01003900648BF83F0200343F46F
:10326800004343F08003484A9BB213602B8856E71B
:10327800116889B2ADF80210BDF80210090414D41F
:10328800BDF802301A067FF579AF627A930003F130
:10329800804303F5B84306EB82021968906948F643
:1032A8000F720A401A60804768E7116840F68F700D
:1032B800013B014056F8233011609847E0E7637BF3
:1032C800013BDBB26373637B03F0FF02002B7FF4E7
:1032D80030AF2F4908684FF6EF73034006200B60A4
:1032E8002073226125E72A4A13689BB243F0100332
:1032F80005200A211360207361731AE7637B013B81
:10330800DBB26373637B002B7FF413AF0423237357
:103318000FE702220323627323730AE71C4D2A680E
:103328004FF6FB7313402B60FFF7CEFE4FF41641A8
:1033380004220123296022732361FAE62369002B02
:1033480000F0828005232373F3E62B88E7E63A68CA
:103358000E4E48F60F731A4033683A601A7A022AFA
:1033680000F08080042A7DD0062A00F0BD80082263
:103378001A7258E7445C004038160020F01B002001
:10338800380000206C930008005C0040EC15002019
:10339800405C00403B689049904E914A40F68F70DF
:1033A80003403B600968336889B221F007010A4489
:1033B800197A52000929126842D092B2520002F1D9
:1033C800804202F5C0421178197092F8018083F8A2
:1033D80001809088C1B2090241EA10215980108900
:1033E800C1B2090241EA102199809289DA8001214B
:1033F8001972002A3CD0B8F1060F00F0D680B8F157
:10340800000F7DD1598831B95A6822F47F42B2F54C
:10341800003F00F02282734F3B6840461B69984783
:10342800032833687ED01A8A4FF6FF718A4279D012
:1034380002284CD108221A72F5E60623237378E68F
:10344800DA8893F80180D2E7674D2A684FF6FB7354
:1034580013402B60FFF738FE4FF4164206232A600C
:10346800237366E6FFF74AFD33681A7A1A72DAE6BA
:103478001A7812F07F0258D1B8F1090F00F01382C0
:10348800B8F1050F00F0A581B8F1030F00F0B38182
:10349800B8F1010F00F0CE81524F3B6840465B699E
:1034A8009847032800F01882336800287FF45FAF3C
:1034B80049494E4A096889B221F007010A44520075
:1034C800002010603021062261801A72ABE6002AC3
:1034D800B0D093F900100029C0F2488103214FF4BD
:1034E80040521972A2809EE65A78052A00F003819C
:1034F8003C4B1B689B689847336808221A7292E60F
:10350800B8F1080F40F0CA801A78500683D1384ABB
:103518009A6100205882904733681A8A4FF6FF71E3
:103528008A42D4D109221A727DE6012A00F02D813F
:10353800022AB1D1B8F1010F00F08881B8F1030F68
:10354800AAD1587947B220F08000820002F1804168
:1035580001F5B841002F0968B4BF01F0300101F44A
:103568004051032898D85888002895D1002993D02D
:103578009B7A002B90D002F1804202F5B842002FCE
:103588001368C0F2E08123F4804323F070039BB2F8
:1035980083F4805343F4004343F080031360154BD6
:1035A8001B689B699847336882E71A7857067FF447
:1035B80032AF9A780B4F012A00F08881022A00F076
:1035C8008881032A7FF428AF3A68526A002A9FD17B
:1035D8004FF0060820E700BF505C0040EC150020C3
:1035E800043000200C160020405C0040023000200F
:1035F800550F000810160020D8F81830B8F81070C9
:103608009BB3002F00F09580B8F81420974228BF8C
:1036180017461FFA87F948469847B14AB14B1268CE
:10362800B8F810E0B8F8121092B222F0070213446A
:103638005B00AEEB090E1A6892B27B1C02F10052D5
:1036480002F540521FFA8EF789445B104FEA420296
:10365800A8F81070A8F8129007D052F8041B20F8A8
:10366800021B013BF9D1B8F81070002F68D0002177
:103678004FF440530846A380FDF78CFDB8F810308E
:10368800B8F81420D6F8008030219A42618053D9C6
:10369800002B5BD0052388F80830C2E5B8F10A0F83
:1036A8007FF4B9AE1A7802F07F02012A7FF4B3AE34
:1036B8009A7A002A3FF4AFAE598800297FF4ABAE5E
:1036C8005A68894F22F47F42B2F5803F7FF4A4AE56
:1036D80058793B689B6998473368002800F0408117
:1036E80093F8018098E6804B1B68DB689847D6F80A
:1036F8000080082395E51A7812F07F027FF4F8AE6F
:1037080093F803C0794840F60F7E036842EA010740
:1037180003EA0E0301323B43042A40F8043BF4D188
:103728007349744A4CF080030B6013681B6A98470E
:10373800DEE6B8F814304BB9032388F8083070E592
:10374800B8F81430D6F80080002BF5D0644A062368
:1037580088F808301168684A89B221F007010A44DC
:10376800520000203021106061805AE5D98801910B
:103778000198824251D95C4A01991268198292F8DB
:103788002C109982FFF7BAFB4DE5B8F10B0F7FF4C7
:1037980083AE554FD9783A68587993699847336812
:1037A8009A7A002A3FF479AE00287FF476AE1A7927
:1037B800002A7FF472AE9B78002B7FF46EAE4D4BDF
:1037C8001B68DB68984733685979DA78D9721A73B5
:1037D8006EE693F90320002AFFF6C9AD9A78002A0D
:1037E8007FF4C5AD9A88002A7FF4C1AD9A7A002A81
:1037F8003FF45EAEBBE5DA78012A7FF44DAE9A88D5
:10380800002A7FF449AE5A7A3A4942F02002096800
:103818005A72CB69984733684AE6914240F28180F0
:103828003149096891F82C60B1B291426FD90022F0
:103838002270A6E7DA78012A7FF42EAE9A88002A49
:103848007FF42AAE5B7A9B067FF526AE04F04CFD2A
:1038580000287FF421AE33682AE693F8008018F038
:103868007F084DD0B8F1010F60D0B8F1020F4BD1ED
:1038780093F8058008F00F018A0002F1804202F5F2
:10388800B84218F0800F126814BF02F0300202F438
:103898004052032938D818F0700835D1002A3FF46F
:1038A800BAAD164A34E6DA788A423FF6F5AD997829
:1038B80000297FF4F1AD998800297FF4EDAD0D4919
:1038C8009A720B685B6898473368F1E53A68D26981
:1038D8007CE63A68126A79E6336809221A72A2E429
:1038E800505C0040043000200C160020005C0040B2
:1038F8004C5C00401016002002300020A10E000889
:103908009A88002ACDD086E54FF0000883E592FB1F
:10391800F6F006FB1022002A7FF433AF0122227052
:103928002FE7104A126892F82C102AE70D4F5879A1
:103938003B689B699847336800287FF4D1AE9A7A30
:10394800002AAED1CCE623F4E04323F040039BB237
:1039580083F0100343F4004343F0800313601EE632
:10396800014AD5E50C1600202D0F0008FF207047EE
:10397800012380F845307047014B1868704700BF35
:103988004C16002001207047704700BF704700BFE9
:1039980008B103487047034B1B6808221A82704716
:1039A8008C000020EC1500202DE9F04190F84450DF
:1039B800002280F8442015B90120BDE8F081184E96
:1039C800736813B91846BDE8F0817368052B02D0F7
:1039D8001046BDE8F081134FD7F8008000F130049D
:1039E800B3682946204683B9FFF720FB3B68A3EB61
:1039F8000803322BA5EB000504440BD8002DDBD0BF
:103A0800B36829462046002BEED03B68A3EB080399
:103A1800322BE5D9B5FA85F04009BDE8F08100BF41
:103A28004C16002040170020002280F84520BBE7F4
:103A380090F844305A1C0344D2B280F8442083F8EA
:103A4800301090F845300BB1132A00D9ACE7704715
:103A58002DE9F041DFF84C80D8F804300BB9BDE807
:103A6800F081D8F80430052BF9D10D4E002A144600
:103A78003768F4DD0D460AE0FFF7D8FA3368DB1B38
:103A8800322BA4EB00040544E9D8002CE7DDD8F874
:103A9800083021462846002BEED00020EEE700BF74
:103AA800401700204C1600202DE9F041234C244EED
:103AB80082B02368002B3AD12568EFB2002D39D0A7
:103AC8000023207B1A46E11801440DF1080E01334A
:103AD8007244DBB2097C02F8041CAB421A46F2D3EA
:103AE80023685B1B2360D4F8008038442073B8F146
:103AF800000F06D0002DDCD09DF8040002B0BDE810
:103B0800F08140210320FDF721FB336884F80C8005
:103B180023F4804323F070039BB283F4405343F4AF
:103B2800004343F080033360002DC2D0E4E701274F
:103B38003D46C5E7207B2F46D2E700BF4C16002044
:103B48000C5C00402DE9F04F87B00A23BE4DBF4FF3
:103B5800BF4CC04E04900393BF4B93F85010986D20
:103B6800C1F3400101F00EF9BB4B93F85010586DAA
:103B7800C94301F0010101F005F905230293B64B91
:103B8800DFF8D892986D01F0EAF8B34B586D01F060
:103B9800E6F84FF0320A4FF0100C4FF47A70D9F86B
:103BA8000430C3F30803002B40F0CB81EFF31183FB
:103BB800002B40F0C6812968A26800BF2B68994293
:103BC800F9D1D7F800E000FB0EF39B1AB3FBFEF324
:103BD80000FB01314FF0010E0191D9F80430C3F315
:103BE8000803002B40F03C81EFF31183002B40F0D9
:103BF80037812B68A16800BF2A689342F9D1D7F8AA
:103C080000B000FB0BF2521AB2FBFBF200FB0323DD
:103C1800019A9B1AB3F57A7FDFD3BAF1010ABED1B4
:103C28008D4BDFF83892986D01F099F88A4B586DF2
:103C380001F095F84FF0320A4FF0100C4FF47A70FB
:103C4800D9F80430C3F30803002B40F05D81EFF38B
:103C58001183002B40F058812A68A16800BF2B68A7
:103C68009A42F9D1D7F800E000FB0EF35B1AB3FBD8
:103C7800FEF300FB02324FF0010E0192D9F8043036
:103C8800C3F30803002B40F0C380EFF31183002B2C
:103C980040F0BE802B68A16800BF2A689342F9D122
:103CA8008846396800FB01FBABEB0808B8FBF1F864
:103CB80000FB0383019A9B1AB3F57A7FDED3BAF12E
:103CC800010ABDD1029B013B13F0FF0302937FF46D
:103CD80056AFDFF888A14FF4FA784FF0100C4FF484
:103CE8007A70DAF80430C3F30803002B40F04681F9
:103CF800EFF31183002B40F041818E462A68A168BA
:103D080000BF2B689A42F9D10B4671469E4600FBCC
:103D180001F3A3EB0E0EBEFBF1F100FB02124FF014
:103D2800010E0192DAF80430C3F30803002B40F0C7
:103D3800CF80EFF31183002B40F0CA802B68A16875
:103D480000BF2A689342F9D18946396800FB01FB14
:103D5800ABEB0909B9FBF1F900FB0393019A9B1A34
:103D6800B3F57A7FDED3B8F10108BAD1049BFF2BF3
:103D780040F03E814FF47A7ADFF8E09050464FF0F9
:103D8800100CD9F80430C3F30803002B40F013815A
:103D9800EFF31183002B40F00E812968A26800BF61
:103DA8002B689942F9D1D7F800E000FB0EF39B1A73
:103DB800B3FBFEF300FB01314FF0010E0191D9F87E
:103DC8000430C3F30803002B66D1EFF31183002BF3
:103DD80062D12B68A16800BF2A689342F9D1D7F84D
:103DE80000B000FB0BF2521AB2FBFBF200FB0323FC
:103DF800019A9B1AB3F57A7FE1D3BAF1010AC0D1CF
:103E0800039B013B03937FF4A7AE07B0BDE8F08F97
:103E1800EFF311818CF31288A2682368DB0344BF97
:103E2800C6F800E0A2682B68D6F80080C9B281F312
:103E380011883968434400FB01F8A8EB0208B8FB75
:103E4800F1F800FB038335E74017002044170020F2
:103E580010E000E03C1700204C16002000ED00E0C8
:103E6800EFF311888CF31288A1682368DB0344BF41
:103E7800C6F800E0A1682B6832685FFA88F888F312
:103E88001188D7F800801A4400FB08F35B1AB3FBCB
:103E9800F8F300FB0233BBE6EFF311888CF31288CA
:103EA800A1682368DB0344BFC6F800E0A1682B685B
:103EB80032685FFA88F888F31188D7F800801A44C6
:103EC80000FB08F35B1AB3FBF8F300FB02338FE740
:103ED800EFF311818CF31288A2682368DB0344BFD7
:103EE800C6F800E0A2682B68D6F80090C9B281F342
:103EF800118839684B4400FB01F9A9EB0209B9FBA9
:103F0800F1F900FB039329E7EFF311818CF3128891
:103F1800D4F808E02368DA0303D501233360D4F822
:103F280008E02B683268C9B281F3118839681A44ED
:103F380000FB01F3A3EB0E03B3FBF1F300FB02322A
:103F480099E6EFF311828CF31288D4F808E023681D
:103F5800D90303D501233360D4F808E02B6831680E
:103F6800D2B282F311883A68194400FB02F3A3EB3A
:103F78000E03B3FBF2F300FB01312BE6EFF31181E3
:103F88008CF31288D4F808E02368DA0303D50123F8
:103F98003360D4F808E02B683268C9B281F311881D
:103FA80039681A4400FB01F3A3EB0E03B3FBF1F3EA
:103FB80000FB0232B3E6EFF311828CF31288D4F8D7
:103FC80008E02368D90303D501233360D4F808E057
:103FD8002B683168D2B282F311883A68194400FB21
:103FE80002F3A3EB0E03B3FBF2F300FB0131E3E6AC
:103FF800954B93F85010986DC1F3400100F0C2FE44
:10400800914B93F85010586DC94301F0010100F02D
:10401800B9FE049BCDF80880013305938A4BDFF87D
:104028002C92986D00F09BFE874B586D00F097FE20
:104038004FF0FA0A4FF0100C4FF47A70D9F80430A8
:10404800C3F30803002B40F0E280EFF31183002B49
:1040580040F0DD802968A26800BF2B689942F9D139
:10406800D7F800E000FB0EF39B1AB3FBFEF300FB4E
:1040780001314FF0010E0191D9F80430C3F3080360
:10408800002B40F08B80EFF31183002B40F08680EB
:104098002B68A16800BF2A689342F9D1D7F800B00D
:1040A80000FB0BF2521AB2FBFBF200FB0323019A4E
:1040B8009B1AB3F57A7FDFD3BAF1010ABED1624BFE
:1040C800DFF88891986D00F04AFE5F4B586D00F05C
:1040D80046FE4FF0FA0A4FF0100C4FF47A70D9F8F8
:1040E8000430C3F30803002B74D1EFF31183002BC2
:1040F80070D12968A26800BF2B689942F9D1D7F816
:1041080000E000FB0EF39B1AB3FBFEF300FB01314A
:104118004FF0010E0191D9F80430C3F308030BBB2B
:10412800EFF31183F3B92B68A16800BF2A689342A3
:10413800F9D1D7F800B000FB0BF2521AB2FBFBF230
:1041480000FB0323019A9B1AB3F57A7FE3D3BAF1F4
:10415800010AC4D1029B059A01339A4202937FF463
:104168005DAF07E6EFF311888CF31288A168236826
:10417800DB0344BFC6F800E0A1682B6832685FFA29
:1041880088F888F31188D7F800801A4400FB08F3F0
:104198005B1AB3FBF8F300FB0233D3E7EFF31188A4
:1041A8008CF31288A1682368DB0344BFC6F800E0DB
:1041B800A1682B6832685FFA88F888F31188D7F805
:1041C80000801A4400FB08F35B1AB3FBF8F300FB0A
:1041D80002336CE7EFF311828CF31288D4F808E00D
:1041E8002368D90303D501233360D4F808E02B688A
:1041F8003168D2B282F311883A68194400FB02F39D
:10420800A3EB0E03B3FBF2F300FB013180E7EFF3FE
:1042180011828CF31288D4F808E02368D90303D5F7
:1042280001233360D4F808E02B683168D2B282F3F6
:1042380011883A68194400FB02F3A3EB0E03B3FBA1
:10424800F2F300FB013114E74C16002000ED00E00A
:1042580010B5FDF777F901280CD14FF4302400E0B0
:104268004CB1FDF76FF9012804F1FF34F8D0002CA8
:1042780008BF052010BD052010BD00BF1A232B2242
:10428800837219230370027300232A220375827034
:104298008375704700231F22027043708370C370B8
:1042A800704730B50446C06C61710368A26823F09A
:1042B8000103036087B0A379009213F004023DD094
:1042C8004FF4805213F00203019244D102934FF449
:1042D80080630022039311F00103059237D1049300
:1042E80008238D07694648BF0493FDF72FFB6079C3
:1042F800E36CA17900F00202002A15BF4FF44032A6
:104308004FF480324FF40034002410F0010F586845
:1043180008BF2246CC074CBF024320EA02025A607B
:104328009A6809074CBF42F0080222F008029A6016
:104338001A6842F001021A6007B030BD13F0020398
:1043480001920BD04FF4005513460295C1E70423A0
:1043580004930C23C5E74FF40053B7E70293B8E77B
:1043680010B50446C06CA160036823F00103036024
:10437800A37986B013F00402009141D04FF4805223
:1043880013F00203019244D102934FF480636279DF
:104398000393D1074FF000030493059345BF04230B
:1043A800049308230C236946920748BF0493FDF73A
:1043B800CDFA6079E36CA17900F00202002A15BFFA
:1043C8004FF440324FF480324FF40034002410F0A0
:1043D800010F586808BF2246CC074CBF024320EAA9
:1043E80002025A609A6809074CBF42F0080222F09C
:1043F80008029A601A6842F001021A6006B010BDFD
:1044080013F00203019207D04FF4005113460291B2
:10441800BDE74FF40053B7E70293B8E770B4EFF382
:104428001186502383F31288436B1A68D20720D46D
:104438005D686DB9446A826A944217D081691144F3
:10444800D9600ED9A21A5A608462002280F85020DE
:104458001A6842F00102F1B21A6081F3118870BC47
:10446800704701698A1A5A608562EEE7012380F86D
:104478005030F1B281F3118870BC704703682DE9A0
:10448800F041DF691FB13B46BDE8F0411847002AFB
:10449800164611DD04460D460E4400E023689B686D
:1044A800204698470028F9D0236815F8011B1B6897
:1044B80020469847AE42F1D1BDE8F08110B5040915
:1044C800013C052C17D80D4B33F8142000F00F00D1
:1044D80042FA00F313F001030DD0012303FA00F0B0
:1044E8000138104002F08AFD054A064B125D10445F
:1044F80003EBC00010BD002010BD00BF6093000892
:1045080058930008441400202DE9F04F4A484B4BBB
:104518004B4C4FF090414FF0010A4FF002094FF019
:1045280004084FF0080C4FF0100E20274026802575
:1045380030F8022B12F0010F03D01960A3F804A081
:10454800083312F0020F03D01960A3F8049008335F
:1045580012F0040F03D01960A3F80480083312F096
:10456800080F03D01960A3F804C0083312F0100F25
:1045780003D01960A3F804E0083312F0200F02D02A
:1045880019609F80083312F0400F02D019609E8096
:10459800083312F0800F02D019609D80083312F49E
:1045A800807F05D04FF4807B1960A3F804B00833EE
:1045B80012F4007F05D04FF4007B1960A3F804B013
:1045C800083312F4806F05D04FF4806B1960A3F89C
:1045D80004B0083312F4006F05D04FF4006B196073
:1045E800A3F804B0083312F4805F05D04FF4805B61
:1045F8001960A3F804B0083312F4005F05D04FF433
:10460800005B1960A3F804B0083312F4804F05D09A
:104618004FF4804B1960A3F804B00833D20B04D0D0
:104628004FF4004219609A80083301F58061A14275
:104638007FF47EAFBDE8F08F60930008441400203B
:1046480000180048002867D003682DE9F04F03F1EF
:1046580038445C4EA40A0125345D04F01F06640941
:10466800022C05FA06F558D0032C00F0A580012C81
:1046780058D08088B0FA80F4C4F11F04A4B2E508C9
:1046880003EB850504F007042E6AA4000F27A74052
:1046980026EA07062E622E6A01F00307A2407C1E56
:1046A8003243012CC1F3810CC1F300182A62C1F313
:1046B80041113CD9C60700F18980850700F1958032
:1046C800440700F1A380020700F1B180C60600F19B
:1046D800BF80850600F1CD80440600F1DB8002062C
:1046E80000F1E980C60500F1F780850500F1058134
:1046F800440500F11381020500F12181C60400F18F
:104708002F81850400F13D81440400F14B810204AE
:1047180000F15981BDE8F08F70472B4CA6693543ED
:10472800A561A6E7284C666935436561A1E70024C1
:1047380022464FF0010E4FF0030904E00132102A1F
:1047480004F10204E6D00EFA02F636EA0005F5D1C5
:10475800D3F808A009FA04F5ED430AEA050AC3F8F4
:1047680008A0D3F808B00CFA04FA4AEA0B0AC3F80E
:1047780008A0B3F804A01FFA8AFA2AEA06069E805F
:10478800B3F804A008FA02F646EA0A06B6B29E8012
:104798001E682E401E60D3F800A007FA04F646EA09
:1047A8000A061E60D3F80CA001FA04F605EA0A0A04
:1047B80046EA0A05DD60C1E7034CE6693543E56171
:1047C80057E700BFF8920008001002401A6822F06C
:1047D80003021A601A683A431A60DA6822F0030280
:1047E8000A438507DA607FF56BAF1A6822F00C027E
:1047F8001A601A6842EA87021A60DA6822F00C0224
:1048080042EA81024407DA607FF55DAF1A6822F058
:1048180030021A601A6842EA07121A60DA6822F04F
:10482800300242EA0112DA6002077FF54FAF1A68D8
:1048380022F0C0021A601A6842EA87121A60DA681F
:1048480022F0C00242EA8112C606DA607FF541AF63
:104858001A6822F440721A601A6842EA07221A603B
:10486800DA6822F4407242EA01228506DA607FF5AE
:1048780033AF1A6822F440621A601A6842EA872243
:104888001A60DA6822F4406242EA81224406DA6059
:104898007FF525AF1A6822F440521A601A6842EA76
:1048A80007321A60DA6822F4405242EA0132DA60CA
:1048B80002067FF517AF1A6822F440421A601A6898
:1048C80042EA87321A60DA6822F4404242EA8132C8
:1048D800C605DA607FF509AF1A6822F440321A601B
:1048E8001A6842EA07421A60DA6822F4403242EA59
:1048F80001428505DA607FF5FBAE1A6822F4402292
:104908001A601A6842EA87421A60DA6822F440227A
:1049180042EA81424405DA607FF5EDAE1A6822F476
:1049280040121A601A6842EA07521A60DA6822F4DA
:10493800401242EA0152DA6002057FF5DFAE1A68DA
:1049480022F440021A601A6842EA87521A60DA684A
:1049580022F4400242EA8152C604DA607FF5D1AE01
:104968001A6822F040721A601A6842EA07621A60EE
:10497800DA6822F0407242EA01628504DA607FF563
:10498800C3AE1A6822F040621A601A6842EA876267
:104998001A60DA6822F0406242EA81624404DA600E
:1049A8007FF5B5AE1A6822F040521A601A6842EADA
:1049B80007721A60DA6822F0405242EA0172DA603D
:1049C80002047FF5A7AE1A6822F040421A601A68FE
:1049D80042EA87771F60DA6822F0404242EA817132
:1049E800D960BDE8F08F002852D0036803F138423F
:1049F8002DE9F04F920A514DAA5C02F01F055209A9
:104A08000124022A04FA05F443D0032A00F0908016
:104A1800012A43D001F003077A1E012AC1F3810C51
:104A2800C1F300188088C1F341113CD9C60700F1D1
:104A38008980850700F19580440700F1A38002076B
:104A480000F1B180C60600F1BF80850600F1CD8077
:104A5800440600F1DB80020600F1E980C60500F19A
:104A6800F780850500F10581440500F113810205F1
:104A780000F12181C60400F12F81850400F13D81F8
:104A8800440400F14B81020400F15981BDE8F08F24
:104A980070472B4A95692C439461BBE7284A5569AE
:104AA8002C435461B6E7002422464FF0010E4FF024
:104AB800030904E00132102A04F10204E6D00EFAD8
:104AC80002F636EA0005F5D1D3F808A009FA04F58C
:104AD800ED430AEA050AC3F808A0D3F808B00CFAAF
:104AE80004FA4AEA0B0AC3F808A0B3F804A01FFAAC
:104AF8008AFA2AEA06069E80B3F804A008FA02F6A3
:104B080046EA0A06B6B29E801E682E401E60D3F89A
:104B180000A007FA04F646EA0A061E60D3F80CA0BD
:104B280001FA04F605EA0A0A46EA0A05DD60C1E761
:104B3800034AD5692C43D4616CE700BFF89200089A
:104B4800001002401A6822F003021A601A683A43F9
:104B58001A60DA6822F003020A438507DA607FF5F3
:104B68006BAF1A6822F00C021A601A6842EA8702D0
:104B78001A60DA6822F00C0242EA81024407DA601D
:104B88007FF55DAF1A6822F030021A601A6842EAAF
:104B980007121A60DA6822F0300242EA0112DA607B
:104BA80002077FF54FAF1A6822F0C0021A601A6830
:104BB80042EA87121A60DA6822F0C00242EA8112D9
:104BC800C606DA607FF541AF1A6822F440721A60AF
:104BD8001A6842EA07221A60DA6822F4407242EA46
:104BE80001228506DA607FF533AF1A6822F4406245
:104BF8001A601A6842EA87221A60DA6822F4406268
:104C080042EA81224406DA607FF525AF1A6822F469
:104C180040521A601A6842EA07321A60DA6822F4C7
:104C2800405242EA0132DA6002067FF517AF1A688D
:104C380022F440421A601A6842EA87321A60DA6837
:104C480022F4404242EA8132C605DA607FF509AFB4
:104C58001A6822F440321A601A6842EA07421A6057
:104C6800DA6822F4403242EA01428505DA607FF5CB
:104C7800FBAE1A6822F440221A601A6842EA874298
:104C88001A60DA6822F4402242EA81424405DA6076
:104C98007FF5EDAE1A6822F440121A601A6842EAEB
:104CA80007521A60DA6822F4401242EA0152DA60C6
:104CB80002057FF5DFAE1A6822F440021A601A680E
:104CC80042EA87521A60DA6822F4400242EA8152C4
:104CD800C604DA607FF5D1AE1A6822F040721A6015
:104CE8001A6842EA07621A60DA6822F0407242EAF9
:104CF80001628504DA607FF5C3AE1A6822F040626B
:104D08001A601A6842EA87621A60DA6822F040621A
:104D180042EA81624404DA607FF5B5AE1A6822F08F
:104D280040521A601A6842EA07721A60DA6822F07A
:104D3800405242EA0172DA6002047FF5A7AE1A68AF
:104D480022F040421A601A6842EA87771F60DA68E0
:104D580022F0404242EA8171D960BDE8F08F30B15B
:104D680002688388918A0B4218BF1B0493617047BD
:104D780010B1036882881A85704710B10368828869
:104D88009A61704738B100298388026814BF0021EE
:104D980010218B409361704710B4094B094A1C7865
:104DA80001238340234052F8200029B9B3FA83F144
:104DB80049095DF8044BE5E7191C18BF0121F8E71C
:104DC8009C160020A01600202DE9F0410B4E3468F7
:104DD80073691C400FD0DFF828800127B4FA84F3E8
:104DE800C3F11F0307FA03F558F82300036898472F
:104DF800AC437561F2D1BDE8F08100BF0004014009
:104E0800AC1600202DE9F0410B4E346873691C4044
:104E18000FD0DFF828800127B4FA84F3C3F11F0309
:104E280007FA03F558F8230003689847AC437561FF
:104E3800F2D1BDE8F08100BF00040140AC160020AB
:104E48002DE9F0410B4E346873691C400FD0DFF830
:104E580028800127B4FA84F3C3F11F0307FA03F586
:104E680058F8230003689847AC437561F2D1BDE850
:104E7800F08100BF00040140AC1600202DE9F0418C
:104E88000B4E346873691C400FD0DFF82880012767
:104E9800B4FA84F3C3F11F0307FA03F558F82300A3
:104EA80003689847AC437561F2D1BDE8F08100BF53
:104EB80000040140AC1600202DE9F0410B4E346887
:104EC80073691C400FD0DFF828800127B4FA84F3F7
:104ED800C3F11F0307FA03F558F82300036898473E
:104EE800AC437561F2D1BDE8F08100BF0004014018
:104EF800AC1600202DE9F0410B4E346873691C4054
:104F08000FD0DFF828800127B4FA84F3C3F11F0318
:104F180007FA03F558F8230003689847AC4375610E
:104F2800F2D1BDE8F08100BF00040140AC160020BA
:104F38002DE9F0410B4E346873691C400FD0DFF83F
:104F480028800127B4FA84F3C3F11F0307FA03F595
:104F580058F8230003689847AC437561F2D1BDE85F
:104F6800F08100BF00040140AC1600200D490E4B33
:104F78008A6942F0010210B58A611A680B4C42F442
:104F880000621A601A6842F480521A602046402271
:104F9800002104F00EF94FF0FF332364C4F84330C6
:104FA80010BD00BF0010024000000140AC160020F8
:104FB8002DE9F041044618460D461646984602F07B
:104FC80015F82768E6722844A07229467D69434689
:104FD80032462046AC46BDE8F04160472DE9F0472F
:104FE8003E4ADFF800E13E484FF00A0C10254FF426
:104FF8007A740127DEF80430C3F30803002B50D17C
:10500800EFF31183002B4CD15668816800BF5368B9
:105018009E42F9D1D2F8088004FB08F35B1AB3FB6F
:10502800F8F304FB063ADEF80430C3F30803EBB9DF
:10503800EFF31183D3B95368D0F8088000BF5168E3
:105048008B42F8D1D2F8089004FB09F1A1EB0808CB
:10505800B8FBF9F804FB0383A3EB0A03B3F57A7FE3
:10506800E1D3BCF1010CC5D1BDE8F087EFF311889D
:1050780085F3128886680368DB0344BF1760866877
:10508800516813685FFA88F888F31188D2F80880A5
:105098000B4404FB08F1891BB1FBF8F104FB031373
:1050A800DAE7EFF3118185F31288D0F808800368F6
:1050B800DE0344BF1760D0F8088053681668C9B289
:1050C80081F3118891681E4404FB01F3A3EB0803E4
:1050D800B3FBF1F304FB063AA5E700BF3C17002039
:1050E80010E000E000ED00E02DE9F0473E4ADFF86F
:1050F80000E13E484FF0190C10254FF47A7401274F
:10510800DEF80430C3F30803002B50D1EFF311830A
:10511800002B4CD15668816800BF53689E42F9D174
:10512800D2F8088004FB08F35B1AB3FBF8F304FB1E
:10513800063ADEF80430C3F30803EBB9EFF3118342
:10514800D3B95368D0F8088000BF51688B42F8D1B2
:10515800D2F8089004FB09F1A1EB0808B8FBF9F8AC
:1051680004FB0383A3EB0A03B3F57A7FE1D3BCF115
:10517800010CC5D1BDE8F087EFF3118885F31288DB
:1051880086680368DB0344BF176086685168136844
:105198005FFA88F888F31188D2F808800B4404FB7A
:1051A80008F1891BB1FBF8F104FB0313DAE7EFF30D
:1051B800118185F31288D0F808800368DE0344BFA4
:1051C8001760D0F8088053681668C9B281F311884F
:1051D80091681E4404FB01F3A3EB0803B3FBF1F34E
:1051E80004FB063AA5E700BF3C17002010E000E0EA
:1051F80000ED00E02DE9F0473E4ADFF800E13E48C7
:105208004FF0C80C10254FF47A740127DEF80430EB
:10521800C3F30803002B50D1EFF31183002B4CD1BB
:105228005668816800BF53689E42F9D1D2F8088059
:1052380004FB08F35B1AB3FBF8F304FB063ADEF849
:105248000430C3F30803EBB9EFF31183D3B9536800
:10525800D0F8088000BF51688B42F8D1D2F8089086
:1052680004FB09F1A1EB0808B8FBF9F804FB038378
:10527800A3EB0A03B3F57A7FE1D3BCF1010CC5D1E6
:10528800BDE8F087EFF3118885F312888668036814
:10529800DB0344BF17608668516813685FFA88F8B3
:1052A80088F31188D2F808800B4404FB08F1891BA5
:1052B800B1FBF8F104FB0313DAE7EFF3118185F38F
:1052C8001288D0F808800368DE0344BF1760D0F85E
:1052D800088053681668C9B281F3118891681E4422
:1052E80004FB01F3A3EB0803B3FBF1F304FB063A59
:1052F800A5E700BF3C17002010E000E000ED00E04B
:1053080000F01F0240090123022803FA02F30ED01D
:10531800032807D0012800D07047074A51690B437A
:1053280053617047044AD1690B43D3617047024AFD
:1053380091690B43936170470010024030B40C4BE5
:105348000178DA6843780B4CD243C2F30222C2F1E7
:105358000402934060181B0101F01F05012249094E
:10536800DBB2AA4080F8003344F8212030BC7047F3
:1053780000ED00E000E100E0554B2DE9F04303EBC0
:10538800800383B0DC68002C00F08880656D514F85
:105398004FF4807304F5AD7206466868A16004F1A5
:1053A8005A012760E0646161A261E3602361287E9D
:1053B800FFF7A6FFEF68FFB1DFF824E1002371468D
:1053C8004868874201F11C0103D001330C2BF7D147
:1053D8000023C3EBC3030EEB83033F481A694169FB
:1053E8004FF00C0E1143721C416183F818E05A7695
:1053F800E36C27632433A364AF683FB3DFF8E0E0CE
:10540800002271464868874201F11C015ED00132D2
:105418000C2AF7D100221046C2EBC2020EEB820220
:10542800DFF8B4E01769DEF814302C493B43CEF8B6
:1054380014300B27731C53761776EA7E234601F047
:10544800A5FBE36CAA6862632833636494F8590087
:10545800FFF734F8074694F85800FFF72FF895F847
:105468001990804647B10B22731CBA71FB713846FC
:105478004A462E21FFF7E6F8B8F1000F0AD00136A8
:105488000C2388F807604A4688F8063040462E21E3
:10549800FFF7D8F8236B2BB1636B1BB1204603B021
:1054A800BDE8F0832B7FAA7E8DF804209B0900219C
:1054B800012201A88DF805308DF806108DF8072017
:1054C800FFF73CFF204603B0BDE8F083D0B2A3E766
:1054D8003C170020A4930008001002405D690008F2
:1054E8009400002040F2E933104900E0B3B10A8982
:1054F800013B12F0020F9BB2F8D00D4B0B4918700C
:1055080040F2E93300E04BB10A89013B12F0010F88
:105518009BB2F8D0064B1878C0B27047054A538F33
:1055280001339BB25387508FC0B270470038004098
:105538000C3800403C17002010B52DED028B9FED74
:10554800208A20EE088A0446B0EE480A02F0A4FF3A
:10555800F0EE408AB0EE480A02F056FFF7EE007A05
:105568009FED187AF0EE675AE8EE875A0023A36198
:10557800B0EE676AC7EEA56A63612362E361A8EECD
:10558800C76ABDEC028B77EEC07AB6EE007AF8EE09
:10559800005A27EE877A20EE250A27EE267A26EE8D
:1055A800266A66EEA77A20EE260A84ED046AC4ED20
:1055B800017A84ED007A84ED027A84ED030A10BD45
:1055C8007CD9A03EF304353F0B4890F850305BB1CE
:1055D800D0F84833013300E00B4690F85020591CAE
:1055E800002AF9D1C0F84833D0F8443303491B687E
:1055F80001F10A00184700BF3C170020921700204D
:1056080050B1202809D021280ED024280ED02528D2
:105618000ED018280ED0002070470023064803EB50
:10562800830300EB830070470123F7E70223F5E7C4
:105638000323F3E70423F1E7CC930008F0B51C78C3
:10564800002A0CBF4FF0200E4FF0300E5D1C4CB3FB
:1056580000292BDD2E4601E01146AAB116F8017B80
:105668004A1E002FF8D18E1E72B1314604680139E6
:105678004A1C671C002A076084F800E0F6DC1C78E6
:1056880026EAE6714A1C5CB1D21A0368591C01600B
:105698001C70AB1815F8014B002CF6D11846F0BD5C
:1056A8001346FBE7002903DC2346F7E70022EBE774
:1056B8004E1EDAE7F0B40D6800240BE0052B18D86D
:1056C800A0F137030A2B14DC04EB840415F8010B52
:1056D80003EB4404A0F13003DEB2092EA0F1610708
:1056E800F2D9052FA0F14103E8D8A0F157030A2BFE
:1056F800EADD0D601460F0BC704700BF3A4B1A78C1
:105708004AB19A7E19691861012A08D002D3042A7D
:1057180000D8704700225A609A60DA60704770B407
:1057280093F82B20B3F9424093ED1A6AD3ED167A19
:10573800D3ED1B6A93ED153AB3F94050D3ED125AE5
:1057480093ED197ADFED293A93ED184AD3ED174A0C
:1057580003EB420240F6E446128F92B205EE102A9D
:1057680006FB02F2B8EE455A401AC4EB12324FF467
:105778007A7101FB02F292FBF5F202FB00F0A5EE52
:10578800036A83B01A65E5EE276A9A6007EE900A05
:10579800F8EEE77A27EE467AE7EEA35AFCEEC67AE9
:1057A800E6EE446ACDED017AF0EE477ABDF80420C2
:1057B800C3ED1A6AE5EE247A06FB02F2C4EB123254
:1057C800BDEEE57A01FB02F2C3ED1B7A92FBF5F21E
:1057D800C3ED125ADA645A6083ED117A83ED037AC5
:1057E80003B070BC704700BF941A00202FE33E310D
:1057F80070B4334B5A7E012A83B013D00022A3F829
:105808007820A3F87A2093F87E20022A07D1B3F8EB
:105818007A10B3F87820A3F88010A3F8822003B098
:1058280070BC704793F82620D3ED286A93ED234A7D
:10583800D3ED244A93ED297AD3ED277A214C93EDC1
:10584800265AD3ED255A2178A578607803EB4202D1
:1058580001EB4114128F92B206EE102AB8EE466A96
:1058680044F6FB76E6EE046AC0EB003004FB026205
:10587800A6EE247AB2FBF0F2B2FBF5F267EEE67A16
:10588800FCEEE64AA6EEC57A92B2A3F88A20CDEDE0
:10589800014AE6EE257ABDF80410A3F87A2004FB45
:1058A8000161B1FBF0F1B1FBF5F189B283ED287A22
:1058B800C3ED297AA3F88810A3F87810A3E700BFEE
:1058C800941A0020881200200A4BD3F8B01081B136
:1058D80010B4D3F8B8406422002002FB04F25DF84B
:1058E800044BB2FBF1F2C3F8B000C3F8B800A3F858
:1058F800B4207047941A00202D4B93F8BC2012B1A5
:1059080093F8BD2002B970472DE9F043294C22785D
:1059180002F0FF0E002A48D1D3F8C020821A002ACC
:1059280043DB254A25491578D3F8C460DFF8988009
:10593800013D6F0007EB050C01EB4C0C3D4401EBFE
:105948000609BCF8042099F814C001EB4501A8FB2E
:10595800028249882578D208013602FB0CF20844F5
:105968000E2E0244C3F8C460C3F8C02088BFC3F831
:10597800C4E035B112480268217801320029FBD110
:1059880002601048D3F8C820D3F8CC10008A01254B
:105998000023257050604B620B889BB22B430B8011
:1059A80013682B431360BDE8F083BDE8F08300BFA4
:1059B800941A00208C17002090170020BC9400082F
:1059C800841A00209C170020CDCCCCCC70B40F4C8E
:1059D8000F4E054607CC0023AA603446286069604C
:1059E800042200E0A27912F0200F04F1140404D17B
:1059F80001330C2BF6D170BC704703EB830306EB25
:105A080083031B79EB7270BC704700BFE0940008F9
:105A1800CC930008F0B400230C4A03611427022633
:105A28000125522464218360836187704360C360C9
:105A3800436186740580847683720183C0F80320ED
:105A4800C0F80B20C0F81320F0BC7047050405000F
:105A58002DE9F04F7A4D81B0FCF700FDD5F8D44020
:105A68000022C5F8D020002C00F0AA80237D052B49
:105A7800074617D9216A23690B44C31A9342B8BF52
:105A880005F1D4010ADBD8E0137D052B0AD9136A86
:105A980012691344FB1A002B80F2CF8051F8042FAF
:105AA800002AF1D14FF0010B00231E46C5F8D03073
:105AB80098469A4625E0636A2169227DFB1AB3FB62
:105AC800F1F301331FFA83F912FB09F201320136AF
:105AD80092B2B6B2A4F81890E282904507D2BBF110
:105AE800000F02D1B9F1010F64D99046A246D5F84A
:105AF800D030013305EB8302C5F8D030D2F8D4405A
:105B08006CB3A268CAB1B4F81690B9F1000FD2D13B
:105B1800216A3846791A9047E8B195F80831002B80
:105B280058D1227D6762013601324FF00103B6B2C7
:105B38002383E2824FF00109CFE7236A2269FB1A27
:105B4800B3FBF2F31FFA83F9A4F81890B9F1000F28
:105B580027D1E28AC1E7A4F81890E28ABDE7D5F810
:105B6800B020D5F8B830C5F818A101321E44C5F8E0
:105B7800B020C5F8B860BAF1000F28D0DAF82030A4
:105B880095F80821AAF81640FB1ACAF81C30CAF87A
:105B980020709ABBDAF80C30384601B0BDE8F04FF7
:105BA8001847227D12FB09F20132013692B2B6B2D1
:105BB800E28292E7237D062B04BF9046A24696E731
:105BC800D5F8B030C5F818410133C5F8B03001B088
:105BD800BDE8F08FFCF742FC05F586710EC9C01BC5
:105BE800A1EB511183420144024438BF0346C5F872
:105BF8000C11C5F81021C5F8143192E7FCF72EFCFA
:105C0800DAF80C3004469847FCF728FCDAF82C2020
:105C1800DAF82830DAF83010001B9042A3EB53135F
:105C28000344014438BF1046CAF82830CAF8301077
:105C3800CAF82C0001B0BDE8F08F4FF0000B33E735
:105C4800941A00202DE9F0413B4ED6F81C510B2D3B
:105C580055DC002D6EDDD6F8D43098424FD0012D9A
:105C680039D0D6F8D830984249D0022D33D0D6F85A
:105C7800DC30984243D0032D2DD0D6F8E03098423E
:105C88003DD0042D27D0D6F8E430984237D0052DE2
:105C980021D0D6F8E830984231D0062D1BD0D6F85E
:105CA800EC3098422BD0072D15D0D6F8F03098421A
:105CB80025D0082D0FD0D6F8F43098421FD0092DE2
:105CC80009D0D6F8F830984219D00B2D03D1D6F860
:105CD800FC30984213D0D6F8D4404CB3237D017DD4
:105CE8008B420FD3154F00243A4605E052F8043F83
:105CF80053B11B7D8B4207D30134A542F6DA00204D
:105D0800BDE8F0810D4F0024631C9B00191F2A1B5E
:105D180006EB840480463944F8189200013503F0F4
:105D28002EFAC4F8D480C6F81C510120BDE8F081D1
:105D3800024FE9E7CFD0E2E7941A0020681B002061
:105D48000D2838B55DD00B285AD8434B342202FBB6
:105D5800003021B1C36813B1BDE8384072E73F4D48
:105D6800D5F81C41002C4BDDD5F8D43098425AD0D8
:105D7800012C45D0D5F8D830984256D0022C3FD0C7
:105D8800D5F8DC30984252D0032C39D0D5F8E03021
:105D980098424ED0042C33D0D5F8E43098424AD0FB
:105DA800052C2DD0D5F8E830984246D0062C27D0BF
:105DB800D5F8EC30984242D0072C21D0D5F8F030F5
:105DC80098423ED0082C1BD0D5F8F43098423AD0EF
:105DD800092C15D0D5F8F830984236D00A2C0FD0B7
:105DE800D5F8FC30984232D00B2C09D0D5F80031C8
:105DF80098422ED00C2C03D0D5F80431984204D008
:105E080038BD164BD3F81801A3E70C2293001448A9
:105E1800A21A191D014492001844013C03F0AFF97D
:105E2800C5F81C4138BD0022F0E70122EEE7022246
:105E3800ECE70322EAE70422E8E70522E6E7062280
:105E4800E4E70722E2E70822E0E70922DEE70A2280
:105E5800DCE70B22DAE700BFE4010020941A0020F7
:105E6800681B00202DE9F04F83B0484C484F019043
:105E7800019803685B699847002840F08380DFF841
:105E880018914448D9F80430DFF810E1C3F3080347
:105E98004FF00A0A4FF0100C4FF47A75002B3BD1E3
:105EA800EFF31183002B37D10168A26800BF0368A4
:105EB8009942F9D1DEF8006005FB06F39B1AB3FBA3
:105EC800F6F305FB013101260091D9F80430C3F33C
:105ED8000803002B3BD1EFF31183002B37D1036864
:105EE800A16800BF02689342F9D1DEF800B005FB53
:105EF8000BF2521AB2FBFBF205FB0323009A9B1A22
:105F0800B3F57A7FE1D3BAF1010AB1D0D9F80430F8
:105F1800C3F30803002BC3D0EFF311828CF312886C
:105F2800A6682368D90302D501233B60A6680368E5
:105F38003968D2B282F31188DEF80020194405FBD3
:105F480002F39B1BB3FBF2F305FB0131BBE7EFF355
:105F580011888CF31288A1682368DB0344BF3E6074
:105F6800A16803683A685FFA88F888F31188DEF850
:105F780000801A4405FB08F35B1AB3FBF8F305FB32
:105F88000233BBE703B0BDE8F08F00BF10E000E0CC
:105F98003C1700204017002000ED00E044170020C7
:105FA800152303701623C370172383712D234370A1
:105FB8002E2303712F23C371704700231B68FFDE54
:105FC80003685A1C02601970704700232622036078
:105FD8000270272282700122436002718371704728
:105FE800F8B5574C0601A7190546387AFFF788F91E
:105FF8003B7A03F01F015B090122022B02FA01F22E
:1060080078D0032B71D0012B67D0A31901351879EB
:10601800FEF754FAEDB2074610B11223C571837129
:10602800A3195879FEF74AFA10B11323C571837181
:10603800A3199879FEF742FA10B11423C571837138
:10604800A5190E21EA793846FEF7FCFA6879FEF7B9
:1060580035FAEA790E21FEF7F5FAA879FEF72EFA55
:10606800EA790E21FEF7EEFAA359364A934251D047
:10607800354A934259D0354A934240D03444227B22
:10608800002A2FD1012002249A8822F48052120477
:10609800120C9A80998889B241F4805199801A88A3
:1060A80002F4415242F44572024322431A809A880C
:1060B80022F470621204120C42F4E0629A809A8B05
:1060C80022F400621204120C07219A8319821A889A
:1060D80092B242F040021A80F8BD1D4B996A0A43F9
:1060E8009A6292E700200446CEE7194B19690A43E1
:1060F8001A618AE7164BD9680A43DA6085E702F520
:10610800EA32116941F400411161116921F4004139
:106118001161B3E702F56042D16841F48051D16062
:10612800D16821F48051D160A8E702F5EC321169F9
:1061380041F480411161116921F4804111619DE7A9
:106148005C1700200030014000380040003C00404F
:106158000010024010B40B49002301E0272B0CD09B
:1061680011F8132082424FEA430403F10103F5D1E9
:1061780021445DF8044B4878704700205DF8044BD3
:10618800704700BFEC9400082DE9F3410569064605
:106198000F467DBBD0F80080C8F30A0323B3002361
:1061A800D6F800800193FEF753F8042819D1224C41
:1061B800236943F001032361BBB2A8F80030FEF75E
:1061C80047F804282ED108F102030193019B3F0CE4
:1061D8001F80FEF73DF82369042823F0010323619B
:1061E80025D06FF0010505E0FEF732F8042805D048
:1061F8004FF0FF35284602B0BDE8F0810E4C236908
:1062080043F002032361C4F81480236943F0400378
:106218002361FEF71DF82369042823F00203236194
:10622800BDD0E5E7236923F001032361D9E733688B
:1062380004333360DEE700BF00200240F8B50446AF
:106248000D468E180027B54201D12069F8BDE368D4
:10625800591CE160234415F8012B1A720429F2D164
:10626800A1682046FFF790FFE7602061EBE770B573
:10627800448806460D46C4F30B04224600212846EE
:1062880002F097FF33690A4A934209D3094A9342B5
:1062980006D2224628461946BDE8704002F064BF7F
:1062A80023B121462846BDE87040184770BD00BF9D
:1062B800C09B0008FA9B0008024A136823EA000002
:1062C80010607047080C0020002870B51EDB0928F4
:1062D800044620DD012303EB83035B00B0FBF3F2EC
:1062E800092AF8D87BB10E4EB4FBF3F00928CCBFCD
:1062F80057223022A6FB03E5024403FB1044EB08B7
:1063080001F8012BF0D100230B7070BD2D230B7009
:1063180040420131DBE7303001F8010BF3E700BF01
:10632800CDCCCCCC884230B44FF001042ED301FB45
:1063380004F4B0FBF4F58D42F9D284B1AAB901E0B6
:10634800B0FBF4F5092DCCBF572230222A4404FBB8
:10635800150003F8012BB4FBF1F4002CF0D1002256
:106368001A7030BC7047B0FBF4F5092DCCBF37224A
:1063780030222A4404FB150003F8012BB4FBF1F486
:10638800002CF0D100221A7030BC70470546002A54
:10639800EBD1D7E70368591C1A46016012F8021BB3
:1063A8000260587841EA0020704738B50446006812
:1063B800154602F0D9FE22682A44226038BD0368D7
:1063C8005A1C026010B4197003680A0A5C1C046045
:1063D8001A7003680A0C5C1C04601A700368090EC2
:1063E8005A1C026019705DF8044B704703685A1C08
:1063F800026019700368090A5A1C02601970704714
:106408000A44914214D030B40139551E41F2210298
:1064180011F8014F082380EA042004044CBF82EAE3
:1064280040004000013B80B2F7D18D42F0D130BC32
:10643800704770B5154C2378A32B24D16378BE2BF5
:1064480021D1214602224FF6FF70FFF7D9FF104EE7
:10645800023422884AB1A518B54214D2052A12D9A5
:106468002146FFF7CDFF2C46F3E721460222FFF72E
:10647800C7FF0222A118FFF7C3FF41F60F53C31A43
:106488005842584170BD002070BD00BF00F003089D
:106498000000040809B10220704701288CBF0220BF
:1064A800002070470B4B1B68DA78042A06D8598AF3
:1064B80030B1094B53F83200084470470020704748
:1064C80010B4054C04EBC2025DF8044B9288511AD3
:1064D80019827047EC15002054040020064B1B68F5
:1064E8005A8A18B1054B186A104470470349898CB9
:1064F8008A1A1A82704700BFEC1500205404002045
:10650800064B1B685A8A18B1054B986A10447047A5
:106518000349898D8A1A1A82704700BFEC1500203A
:1065280054040020074B1B681B7803F07F03212BC2
:1065380001D00220704700F0DF00022814BF0220BB
:1065480000207047EC150020212804D0202803469D
:1065580011D0022070470F4B1A68137803F07F039D
:10656800212BF6D10C4910B50024916154822046A4
:106578008847204610BD074A1268117801F07F014C
:10658800212903D0054A02201370704703480449A3
:106598000370E8E7EC150020AD650008EE1B00204D
:1065A80099390008FDF7F4B9704700BF034B1A7812
:1065B800202A04BF00221A70704700BFEE1B00207B
:1065C800014B04221A60704750160020034B9B7A37
:1065D80013B1034B05221A60704700BFF015002065
:1065E800501600200D4A0E4B12680E4992B222F046
:1065F800070213445B001B68C3F309030B600B68B5
:106608009BB201335B1007D00749084A52F8040BC4
:1066180021F8020B013BF9D1704700BF505C0040E4
:106628001E3000204C1600205C160020206200401E
:10663800014B00221A607047541600202DE9F04FD4
:106648006A4BDFF8D0811A68694DDFF8CCB1DFF802
:10665800CC9168496848DFF8C8A1684F83B0002426
:10666800C02353729472D4720193C8F800402A6808
:1066780002EA0B0242F4007292B22A602A6802EA25
:10668800090292B248F2800682F0100232432A6070
:10669800D8F8002092B222F00702114449004022A3
:1066A8000A60D8F80010009289B221F0070101F1C0
:1066B800005101F5405149004FF0800EC1F800E04B
:1066C800D5F800E090F82C1040F60F6000EA0E00B4
:1066D800304328602046FAF739FD29684848DFF832
:1066E80044E1019B009A01EA0A0189B281F4405110
:1066F80031432960016801EA0B0189B20160D8F8C9
:10670800001089B221F007018E444FEA4E0E11465F
:10671800CEF8003003683B4ADFF80CE103EA0903CE
:106728009BB283F0200333430360036803EA0A0340
:1067380033439BB203601368334803EA0B0343F403
:10674800C0639BB21360D8F800309BB223F00703F4
:106758009E444FEA4E0E4FF48073CEF80030136813
:1067680003EA0A0333439BB21360136803EA09037D
:106778009BB283F02003334313603B6803EA0B0B9F
:106788001FFA8BF33B60D8F800309BB223F0070365
:10679800184440004FF4887303600320FAF7D6FCCE
:1067A8003B6803EA0A039BB283F4405333433B60DC
:1067B8003B6803EA090333439BB22A4620463B6001
:1067C800314640F60F75136840EA01042B4001304A
:1067D8002343042842F8043BF5D10C490C4B802094
:1067E800012208601A6003B0BDE8F08FEC150020A4
:1067F800005C004004300020380000200C5C0040A1
:10680800045C0040085C00401C3000204C5C0040E8
:1068180050160020505C00408F89FFFFBF8FFFFF9C
:106828008FBFFFFF0830002010300020F8B5134A52
:10683800134B10681B68C0180AD0124B12491C6809
:106848000822FCF727FC204604221049FCF722FC0A
:106858000F4B104A19681048104D114C00238B72C9
:1068680001274FF416414FF4E05617601360036098
:1068780016600360698011602360F8BDACF7FF1FE4
:10688800B4F7FF1FB0F7FF1F86040020960400200E
:10689800EC150020405C0040445C0040EE1B0020EA
:1068A80050160020024B4FF480221A60704700BF38
:1068B80014040140F8B50568037B2A6802269E4047
:1068C80032420DD1296804229A40114218BF6A60E9
:1068D8002968082202FA03F3194218BF6B60F8BD51
:1068E8001749184A0B684FF6FE7423400B6013894A
:1068F8009F07FCD5134B1A891406FCD41B89D907AA
:1069080018D411490F4A0B684FF6FE773B400B60CD
:106918006E60938823F0030304461B040B481B0C8A
:1069280093800068FEF729FA094A2568237B00212D
:106938001170C7E7034B9A891A89D207E1D5FAE79C
:10694800440002400038004058000240B4130020C0
:10695800270C002010B490E80600047B406902234D
:10696800A3404B6013685DF8044B4FF6FE710B4073
:106978001360FDF753BD00BF2DE9F84F294A13787E
:1069880003F0FF04002BFAD1274FDFF8A8803868FE
:10699800DFF8A490254D012388F80030FEF7E8F9C8
:1069A8000520FEF79FFD2046FEF79CFD0620FEF71A
:1069B80099FD2046FEF796FD99F80060042046F000
:1069C8000106FEF78FFD3046FEF78CFD2B8893B14C
:1069D800DFF868A0164E1AF804B00720FEF782FD0B
:1069E8005846FEF77FFD1AF804202B8832550134EB
:1069F800A4B2A342EFD80720FEF774FDFF20FEF7EC
:106A080071FD99F800400420FEF76CFD2046FEF762
:106A180069FD3868FEF7B1F9002388F80030BDE851
:106A2800F88F00BF270C0020B413002000000020BE
:106A38004C0E0020340E00203D0E0020280C0020B3
:106A48002DE9F041474E3068FEF792F9464B1B7826
:106A5800012B78D05FD3022B0AD1DFF82C810823D1
:106A680088F800300D254FF4C373404F3B8010E089
:106A7800DFF814813D4F98F8003003F04003002BF5
:106A880014BF4FF4F0734FF4C3733B8014BF102549
:106A98000D25002404F11000C0B2FEF723FD0134D7
:106AA8000120FEF71FFDA3B2AB42F3D398F80040D4
:106AB8002F4D0020FEF716FD2046FEF713FD2D4B47
:106AC8001C780220FEF70EFD2046FEF70BFD2A4B30
:106AD8001C780320FEF706FD2046FEF703FD274B32
:106AE8001C7804200443FEF7FDFC2046FEF7FAFC60
:106AF8003068FEF742F93A882148002102F059FB34
:106B08002B7833B11F4B1B7833B300232B70BDE8B0
:106B1800F081BDE8F081A020FEF7E4FC0020FEF73C
:106B2800E1FC00F00603022BDFF85C8007D000F0E0
:106B38000500012803D1482388F8003008E008231D
:106B480088F800308EE7DFF84080482388F8003066
:106B580010254FF4F07388E7FFF70EFF00232B7022
:106B6800BDE8F081B4130020B81300200000002015
:106B7800A0040020BF130020C01300203D0E0020F9
:106B88004C0E0020340E00200200002070B50F4C7F
:106B98000F4DC0EBC00004EB8004686926693043E0
:106BA800686182B09209667BA1600025012101A875
:106BB80063618DF804608DF805208DF806508DF816
:106BC8000710FEF7BBFB02B070BD00BF94000020A9
:106BD800001002400348D0F83C3113B100F59A7018
:106BE80018477047940000200348D0F8203113B1AB
:106BF80000F58C7018477047940000200348D0F8BF
:106C080004310BB1FC301847704700BF94000020D6
:106C18000348D0F8E8300BB1E0301847704700BFA0
:106C2800940000200348D0F8CC300BB1C43018478A
:106C3800704700BF940000200348D0F8B0300BB173
:106C4800A8301847704700BF940000200348D0F8C8
:106C580094300BB18C301847704700BF9400002067
:106C68000248836F0BB170301847704794000020BA
:106C78000248C36D0BB15430184770479400002088
:106C88000248036C0BB13830184770479400002055
:106C98000248436A0BB11C30184770479400002023
:106CA8000248836803B11847704700BF940000206A
:106CB8001749184B184A194810B4D1F8884044F4B9
:106CC8007004C1F888401C6844F001041C605C68CA
:106CD80022405A601A6822F0847222F480321A60C4
:106CE8001A6822F480221A605A6822F4FE025A6056
:106CF800DA6A22F00F02DA621A6B002410404FF0B1
:106D0800006218639C608A605DF8044B704700BF9E
:106D180000ED00E0001002400CC07FF8CCFC00FF42
:106D28002DE9F041804B814C1D885B88E278EB1A95
:106D380083EAE3719542A1EBE37149D32378AB422F
:106D480046D37B4A1378DE1E012E40F29D80794E91
:106D58003678022E00F08E80012B6DD077D3022B6F
:106D680004D19188A94201D201231370E17A002944
:106D780048D02189002945D06F4D2D78002D41D06C
:106D88006E4D9FED6F6AD5ED026A07EE901AF8EE28
:106D9800E66AB8EE677AF8EEE77A77EE666A66EE44
:106DA800866A86EEA77AFDEEC77A17EE901A002952
:106DB800C0F29380642900F3B480002900F08D802C
:106DC800C9B2257B8D422CBF0125002555701AE0DC
:106DD800B5EB420FB5DC564A1378DE1E012E40F2A1
:106DE80098800229B3DC534BDFF84CE11F7800266A
:106DF8000323022F8EF8006056809680137053701C
:106E0800B4D139E055782479632C03D8022B117A50
:106E180066D029B9AB4238BF2B461374BDE8F08160
:106E2800D168401A4749884260DDAB4238BF2B46DB
:106E380054721374BDE8F0819188667B891B8D427A
:106E48000CDD5188A94291D2002313708EE7568831
:106E5800637BF61AB54287DD002387E702231370A8
:106E680084E70229BFDD334B1B78022B4FF0040364
:106E78007FF47CAF304E3678334F0229CCBF0021E7
:106E88000121F980BE8067E702293FF760AF2678C5
:106E980095FBF6F6771C082F274BDFF898C0A678E5
:106EA80094F801E09CF800C0A8BF08271F70BBB287
:106EB80016FB03F61EFB03FEB6B200234FF0640870
:106EC800BCF1020F5680A2F804E013705370D3602F
:106ED80082F80980BCD13EB2CEE70225557092E710
:106EE80000299DD10126D06016720846C4F16404B9
:106EF800164900FB04F081FB0041C017A0EBA1502C
:106F0800AB4200F1640038BF2B4650721374BDE8E1
:106F1800F081032BA5D1074E3678022E7FF426AFD9
:106F2800A8E764214DE700BF0C1B0020A81A002029
:106F38005C1C0020121B0020941A0020981A0020C4
:106F48000000C8427F969800141B00206BCA5F6B34
:106F58001F4B204870B53422012500211D7002F016
:106F680028F91D4A1D491E4C1E4800230B6013605A
:106F7800FEF768FE29460520FEF7E2FE6579291C22
:106F88004FF0070018BF0121FEF7DAFEA679311C81
:106F98004FF0080018BF0121FEF7D2FEA37A0BB903
:106FA800E17A19B195B9311C18BF01210920FEF702
:106FB800C7FE0D4B59690A20C1F34051FEF7C0FEC8
:106FC80001210B20BDE87040FEF7BABE0121EDE7B4
:106FD8009C1B0020681B0020B01B0020641B0020A5
:106FE800A81A0020E40100205C1C0020034613F8C6
:106FF800012B002AFBD1181A01387047430803F007
:107008005533C01A830803F0333300F03330184483
:1070180000EB101000F00F3000EB002000EB0040F8
:10702800000E704711481249026800608A4218D061
:10703800002103E00F4B5B58435004310E480F4BBF
:1070480042189A42F6D30E4A02E0002342F8043B63
:107058000C4B9A42F9D3FFF72BFE00F019F8704752
:10706800FEE70948D0F800D040680047FC9F0020A0
:10707800EFBEADDEFA9B000800000020B804002037
:10708800B8040020741D002000D8FF1FFEE7000090
:107098002DE98048C64BC74A9FB01968914200AF96
:1070A80000F03F85C449C54B00224FF47000C1F879
:1070B8008800BA61FA611A6842F480321A6003E003
:1070C800BA69B2F5A04F09D01A6802F40032FA6121
:1070D800BA690132BA61FA69002AF1D0B74B1B6864
:1070E80013F4003318BF0123FB61FB69012B00F087
:1070F800ED84B14CB14BB24AE2605A6A5A6ADFF881
:107108001C9342F080725A625A6942F4FC025A6136
:1071180000250322012307F1280141F6FF764FF0ED
:107128009040FD62BE6287F82C2087F82E30FAF76F
:1071380069FC4FF6FF7307F12801A248BB62FAF712
:1071480061FC07F12801A048A04EFAF75BFC07F1A3
:1071580028019F48FAF756FC07F128019D48FAF7DD
:1071680051FC07F128019C48FAF74CFC07F128006C
:10717800FAF7FCF9BB6A9949994A9A48A1FB0313A3
:107188009B0C3360F0210723506084F8231095602E
:107198001360FDF7B9F9FFF74CF9934D002800F09B
:1071A800A883924CA94523D2DFF87092DFF8708249
:1071B800464633889B46F2188BB1A2420FD2052B64
:1071C8000DD9B9F800307188C3F30B03994200F068
:1071D800D180164633889B46F218002BEDD1D9F89A
:1071E8000410484609F11409FFF741F8A945DFD30F
:1071F800FBF7F6FD002800F0D7800120FFF75CF8C8
:107208000820FFF759F84020FFF756F88020FFF7CD
:1072180053F84FF40070FFF74FF84FF48060FFF712
:107228004BF84FF40050FFF747F84FF48040FFF752
:1072380043F84FF48030FFF73FF84FF40030FFF782
:107248003BF84FF48020FFF737F86948694CDFF8BE
:10725800D491694DDFF8B4A1FFF72EF84FF0007014
:10726800FFF72AF84FF08060FFF726F84FF000602C
:10727800FFF722F84FF00050FFF71EF85F4A604B07
:10728800604910781B78604A08705D481268E17898
:10729800C9F8002043F00103037029704FF0010B77
:1072A8004FF0050814F8010B002840F0E380CAF8F5
:1072B80000000BF1010BBBF1040F0AF1040AF1D134
:1072C8002978524B524C1868C94301F00101FDF767
:1072D80059FD29784D4B81F002015868C1F34001EE
:1072E800FDF750FD2978494B81F004019868C1F3F6
:1072F8008001FDF747FD01210220FDF74DFDFDF757
:1073080035FE6420FBF70CF8FAF770FE2320FDF732
:10731800D5F8C4F8B80418B1112200238271C371DA
:107328000121FDF760FBD4F8B804394CDFF8F8B058
:10733800FDF71EFD374B224619201A21002503F1BF
:10734800110E03F114080BEB050C29B19CF80AA0E7
:107358008A4508BF82F8581028B11BF805108142E9
:1073680008BF82F85900F04560D01EF8011B9EF84E
:107378000300EAE7737999077FF42BAFD9F8041073
:1073880096F804A04846FEF772FFB9F80030BAEB49
:10739800133F5FD009F11409A945FFF409AFFBF7C2
:1073A8001FFD00287FF429AF1B48FEF733FB24E7B5
:1073B800FC9F0020EFBEADDE00ED00E000100240B3
:1073C8000005FA050004004800080048441700209A
:1073D800000C0048001000480014004883DE1B43DE
:1073E80010E000E03F190100C09B000800000408FD
:1073F80020001000F81600209C160020000C002029
:107408009A120020121B0020080C0020A016002051
:10741800B8040020CC910008C81300206C9A00081A
:1074280002F00308701C00201C170020B2F8581046
:1074380029B1C349536541F8252002F51772C1499E
:10744800994227D093F8205093F8301093F83400DD
:10745800203374E7B9F80230D9F80400ABF106021A
:10746800C3F30B039A4206F10601A8BF1A4601F0BE
:107478007BFE8FE7FDF722F80121CAF800005FFACA
:107488008BF320B180F80680C371DAF80000FDF7AD
:10749800AAFA0EE7FBF786FC0020FEF7A1FDDFF84D
:1074A800E4B2A94D0120FEF79BFD4FF0000A2146EA
:1074B800002D48D01BF90B8C39604FEA880303EB89
:1074C800080E7B60A14B03EB0804A14BA27816467B
:1074D8009E4A12F80820FA604FEA8E009C4A03443C
:1074E80042F82EA00A18BA60C3F804A0C3F808A08E
:1074F800C3F80CA0C3F810A0ABF1030414F8012BD7
:10750800FB689A422ED0A278B24224D0A345F5D186
:1075180097E80A00434401EB8303D3F8C40490B10D
:10752800D3F8C80478B1894AC3F8C0549044ABF181
:107538000B0098F8044098F8062083F8CC4483F8A8
:10754800CD24C3F8BC04834B0BF1100B9B4510D022
:107558005BF8075CACE73046FCF7B0FFBB68C3F8E4
:10756800C804D3E71846FCF7A9FFBB68C3F8C404EE
:10757800C9E7D1F8BC340C46002B66D001F59865F4
:1075880095E82005987BFDF7BBFE734B9D4200F004
:107598009E81724A136B23F01003136310216F4A04
:1075A800136B0B431363B8F1000F05D015220123A9
:1075B80088F8062088F8073094F8CD34002B0CBFE3
:1075C8001E213E2140460422FDF73CF8BAF1000F87
:1075D80005D0162201238AF806208AF8073094F885
:1075E800CD34002B0CBF1E213E2150460422FDF74E
:1075F80029F8296894F8CC44594B5A485A4A21F03A
:10760800010129602968002C18BF03460A402A6036
:107618002B612A68002342F001022A60AB60EB600C
:10762800AB60AB6843F40043AB602B682B606B68BE
:1076380023F0784323F400436B602B6823F4003372
:107648002B602B6843F001032B60484B484A9C7918
:107658005D79D9F80000474BA4F10101A5F1010EAD
:10766800B1FA81F14909BEFA8EFE4FEA5E1E012D7C
:1076780011714FF00001196082F800E05960C0F301
:10768800C03E9960D960196100F4004008BF517884
:1076980082F802E008BF197008B1D178D9739179DE
:1076A80009B1D1799972012C08BF5279314D08BFBF
:1076B8005A710023AA4698464FF0070B01249AF8FE
:1076C8000000002840F0CB800BF1010B5FFA8BFB28
:1076D800BBF10B0F0AF1050AF1D1002B40F0DC8059
:1076E800254C01210846FDF757FB00210846FDF708
:1076F80053FB00210220FDF74FFB0A251F4B58685A
:10770800FDF72DFB1D4B1868FDF729FBFDF7ECFC79
:10771800FDF7EAFC013DF1D129462846FDF73CFB7F
:1077280029460120FDF738FB4FF419722946144801
:1077380001F03FFDFBF712FB4FF0CC0A38BB51E0DC
:1077480048170020EC91000800540040D01B00208E
:1077580074090020379200080058004000100240C9
:107768007A25E000300E5000FFE0CF00A81A002074
:1077780098130020B81A002094000020A0160020BA
:107788009C09002017920008D5B2022D2AD80AFBBE
:1077980005F8AF4B53F808306A1C002BF4D1C278B7
:1077A800FB60AC4B90F9020003EB8202116EFBF711
:1077B800D9F8834605EB450000EB0010BBF1000F3C
:1077C8000CD0FB681946A24BCC2203EB800001F0D9
:1077D800F0FC9F4B013543F808B0EDB2FBF784F895
:1077E8000028D2D1FAF7F4FF08B1FAF765F9D9F809
:1077F80000309B0200F1C7819749984D9848994AF3
:10780800994C04230B702B700021984B0180642045
:10781800596019705870964B11805B79954A2170A0
:10782800012B1180518000F0A481914B924A9979E3
:1078380092480023012903701360536093604DD070
:107848008F4B1B68C9F80030FFF782FB8D4B8D4AC0
:107858001B7863F07F031370FEF7FAF8FCE7FCF778
:107868002DFE132118B1002380F806B0C371FDF76F
:10787800BAF89AF80000FEF76DFC072308F1010238
:107888008AF802808AF804308AF801008AF80340EE
:107898005FFA82F8012317E77B4B7C4CDA6A22F403
:1078A800F872DA62DA6A42F4D872DA623C20FDF7DA
:1078B80027FD77482246002303E001330C2B00F014
:1078C800C1835168814202F11C02F6D1BBE36E4AC2
:1078D8007049136B23F02003136360E66E4A9FED33
:1078E8006F0A6F48136053609360D360FDF724FEFE
:1078F800A6E7A94538BF4C4606D26168204614342D
:10790800FEF7B5FCAC42F8D3664A674CDFF8B8819D
:10791800012313813B60654BE31A7B600323BB6043
:107928000026624BBB627B683E637E63BE63FE6378
:10793800FB62D8F81030180606D55D4BC8F804303D
:1079480003F18833C8F804303B7887F83C30A3202B
:107958003423C8F80C300222BE2307F11001387412
:1079680007F128007B74FEF769FC022207F1100179
:107978004FF6FF70FEF744FDA945834633D24D4BC1
:10798800FB60FA6887F82560B2F802A01388CAF38A
:107998000B0AC3F30B000AF106011B0B06223984FC
:1079A800788407F1200107F1280087F82430FEF7D2
:1079B80045FC5846062207F12001FEF721FDFB6829
:1079C80083465968524607F12800FEF737FCFB68E2
:1079D8005846596852461433FB60FEF711FDFB68A0
:1079E800AB428346CDD3022207F1140107F12800E8
:1079F800BE82FEF723FC022207F114015846FEF767
:107A0800FFFC43BADB43022207F1200107F12800FB
:107A18003B84FEF713FC786B002840F09A80B86B23
:107A280097F83C30002B40F08D80002840F084808F
:107A3800FEF7FFFC00287FF4B5AB0520FCF782F8C1
:107A48001D491E4B1E481F4A0860DA60FFF7AABB93
:107A58009C090020CC9100085C1C00206C1C0020B4
:107A6800601C00205E1C0020941A0020641C00206A
:107A7800A81A00200C1B0020981A00205D1C00206A
:107A8800080C00209A1200200010024094000020E8
:107A98000800024020000010D81A0020CDCCCC3EAF
:107AA800E81A0020C81300200000040800F00308AA
:107AB800230167456C9A0008FC9F002000ED00E058
:107AC800EFBEADDE0400FA05002002409E4A9F4B3F
:107AD800122111605A685A605A685A605A6842F40A
:107AE80080625A605A6822F47C125A605A6842F4DA
:107AF800E8125A601A6842F080721A601A68940193
:107B0800FCD55A68914922F003025A605A6842F03B
:107B180002025A604B6803F00C03082BFAD1FFF7F6
:107B2800E8BA00221A6062B6894B1B6883F308889A
:107B3800884B1B689847FEE7BB68013BBB607FF436
:107B4800F0AE7AE7D8F8103043F08003C8F8103068
:107B58006BE707F13003C0F104020021184401F07B
:107B680028FB396B07F12800FEF70EFB7E63B8632C
:107B780056E72822784801F01CFB9FED780A7848E0
:107B8800FDF7DAFC51E6774B93F80BA01B78BAF1B6
:107B9800000F07D0022B00F03B83032B00F02F834C
:107BA800012B09D0704B00221A70704B6F4A1B785A
:107BB80043F0080313701FE66D4D6E486E492B7035
:107BC80018224FF43473C5F8E4026A60A96005F11D
:107BD80014001A4600212B6101F0EBFA5046FDF71C
:107BE8000FFDDFF8B481C3680268F860C8F80020A8
:107BF800002B00F041815046FCF760FC5F4B186099
:107C080018B1292200238271C371FE684E21327A8D
:107C1800FCF718FD307C4D4A59495369C0EBC00E3A
:107C280004EB8E0EDEF81040234353610024292212
:107C380023468EF818208EF81940C022FEF7A6FFBA
:107C4800D8F80000FAF728FBFDF75AFBA8884D4939
:107C58004D4AD8F8003001FB00F1914208DC02EBF4
:107C68005104B4FBF1F4013CA4B2611CB2FBF1F283
:107C780046481988AE68B2FBF6F28342C2F34E0E4C
:107C8800A5F80CE092B289B200F0C98100F5006055
:107C9800834200F0C481B3F1804F00F0C081A0F5A9
:107CA8009830834200F0BB8100F58060834200F089
:107CB800B6813748834200F0AE8100F58060834288
:107CC80000F0A98121F4407100F58C3089B283421B
:107CD8001980DA621C8500F09B812E4A934200F0DD
:107CE800978102F54062934200F0928102F580622A
:107CF800934200F08D8102F58062934200F0888102
:107D08000121FA685961D079FA6810F0040E5279A5
:107D180017BF00244FF4807421464FF0040E00F082
:107D280002000C2A00F25381DFE812F00D01510124
:107D380051015101E600510151015101B2005101B7
:107D480051015101380000BF0020024000100240DC
:107D580000D8FF1F04D8FF1F1C1B0020CDCCCC3D32
:107D6800201B002090170020501B00209A12002092
:107D78009C17002070920008CE0707009C12002074
:107D8800691D000840420F0000A24A04002C01406F
:107D98000010004000340140601B00201A6ADFF820
:107DA8009CA222F480521A621A6AD3F804C0D3F84B
:107DB8001CE022F4005242EA00322EF4E64E53450B
:107DC80042EA01324EF4C04E00F0888096498B4258
:107DD80000F084800021C3F804C0C3F81CE01964D3
:107DE8001A62DA6942F40062DA615A6CFE688F4CF2
:107DF800F06842F400425A64036820604FF6FE724D
:107E080013400360F9F704FA07F12800F9F7D2F9EB
:107E1800D8F8003072792969B98634331344BB62C3
:107E280010228023002507F128012068DFF810E2DE
:107E38003A63FB634FF480724FF40053FB643A6477
:107E4800C7F82CE03D65BD637D64BD64F9F7C0F9F2
:107E58007279D8F800100C2A98BF754BC86896BF7D
:107E680003EB42022B46B2F8AC3022680343CB60E6
:107E7800136843F0020313606E4C01252570FDF76B
:107E8800A3FB2378002B3FF490AE6B4B1D708CE660
:107E98001A6ADFF8A8B122F480721A621A6AD3F853
:107EA80004A0D3F81CC022F4007242EA00222CF08D
:107EB800730C5B4542EA01224CF0600C13D05A491E
:107EC8008B4210D00021C3F804A0C3F81CC0D963AA
:107ED8001A62DA6942F00802DA6186E72CF4804C0B
:107EE8004CEA841C76E722F440622AF4405A42EABB
:107EF8000E224AEA041AE5E71A6ADFF840B122F0CE
:107F080010021A621A6AD3F804A0D3F818C022F033
:107F180020022CF0807C42EA00122CF4E64C5B45EF
:107F280042EA01114CF4C0423FD03F4883423CD062
:107F38000020C3F804A09A61986319629A6942F410
:107F480000629A6151E71A6ADFF8F0B022F0010284
:107F58001A621A6AD3F804A0D3F818C022F00202F1
:107F68002CF4803C02432CF0730C5B4541EA02017F
:107F78004CF0600222D02C4883421FD000F54060AC
:107F880083421BD000F58060834217D000F58060E3
:107F9800834213D00020C3F804A09A615863196281
:107FA8009A6942F008029A611FE721F0C0012AF499
:107FB800406A41EA0E114AEA840AB9E721F00C0145
:107FC8002AF4407A4EEA010144EA0A0AE2E70C2A56
:107FD8003FF60BAF01A151F822F000BFA97F0008BE
:107FE800F37D0008F37D0008F37D0008457F000855
:107FF800F37D0008F37D0008F37D0008DB7E0008B0
:10800800F37D0008F37D0008F37D0008EB7D000890
:1080180000221A8674E61980DA621C8570E621F05F
:10802800700189B245E600BF003401405C1B0020A6
:10803800CC910008501B0020511B0020002C01404F
:10804800B01700200023C3EBC30304EB83039B4951
:108058001E694A699A4832434A614FF0000A06226B
:108068001A7683F819A08346F9F7D2F807F12800A1
:10807800F9F7A0F8B8F1020F34BF534680239149AD
:10808800914AFB63B9624FF480734FF4806158469C
:10809800FA623B6420224FF40053796407F1280107
:1080A800C7F830A0C7F838A0C7F850A0BA64FB6476
:1080B800A7F83480F9F78CF8DBF800304FF0A04AC5
:1080C80043F00103CBF80030DAF8083023F04053CE
:1080D800CAF80830DAF8083043F08053CAF8083094
:1080E800FCF77CFFDAF8083023F08043CAF8083040
:1080F800DAF80830CAF80830DAF8083043F00043F4
:10810800CAF8083053469A68002AFCDB9868DFF8FA
:10811800D4E16E496E4A20F040509860986840F06B
:1081280000509860DEF80800014041F46831CEF84C
:108138000810D9680A4042F40052DA60196B08F155
:10814800FF3221F00F010A431A634FF0A0400123C8
:108158004FF0070B4FF01F0E03E05E4A0535AA42A9
:1081680031D0EA78002AF8D003F1010C042B5FFA29
:108178008CFC95F8018029795ED803EB43035B00FA
:10818800026B0EFA03FA22EA0A0208FA03F313430F
:108198000363B8F1090F5FD808F1FF3342694269F8
:1081A80003EB4303382606FA03F822EA0802426181
:1081B800DA1C436901FA02F21A434261454A05355D
:1081C800AA426346CDD14FF0A0421346916841F0D0
:1081D800010191601A68D207FCD5DA6822F0020220
:1081E800DA60DA6842F00202DA60DA6842F0010224
:1081F800DA609A6842F004029A60FFF772BA364D64
:10820800364BC5F8E4321222C82349F27041DCE447
:10821800314D334BC5F8E432182100234AF29E321F
:108228006960AA6005F114004FF41B7219462B709F
:108238002A6100F0BEFFD1E4092B1FD8053B03EBF0
:1082480043035B00426B0EFA03FA22EA0A0208FAB9
:1082580003F3134343639CE7A8F10A028369836924
:1082680002EB42020BFA02F823EA080383618369EE
:1082780001FA02F21A43826163466EE70E2B0DD8AB
:108288000A3B03EB43035B00826B0EFA03FA22EA14
:108298000A0208FA03F3134383637AE7A3F10F0290
:1082A80002EB42025200C36B0EFA02FA23EA0A03F7
:1082B80008FA02F21343C3636BE700BF00100240E1
:1082C8000800024040000050CC1A0020E010FCFFDB
:1082D80007C0FFFDCC1A00209C17002074920008EC
:1082E8006C9200080003005038B5444B1A681078A7
:1082F80010F07F0004D1537A23F02003537238BD65
:10830800022878D15388002B76D11379002B73D1AA
:10831800537923F08000840004F1804101F5B841CD
:108328005DB20968002DB4BF01F0300101F440517D
:10833800032860D800295ED0927A002A5BD004F125
:10834800804404F5B844002D226824DA02F0300293
:10835800102A4AD103F07F039A0002F1804202F505
:10836800B8421368590608D5136840F60F710B40D8
:1083780043F4004343F0C0031360136823F4E0435D
:1083880023F040039BB283F0300343F4004343F0EF
:108398008003136029E002F44052B2F5805F24D1D3
:1083A80028B9174B93F82C10F8F7D0FE10E09B0073
:1083B80003F1804303F5B8431A68520408D51A68D4
:1083C80040F60F710A4042F4404242F080021A60BF
:1083D800236823F4804323F070039BB283F4405353
:1083E80043F4004343F080032360064B1B685B693A
:1083F8009847002038BD022038BD00BFEC1500208A
:10840800380000201016002000B510EE103A204A5F
:1084180023F00043934283B019DDB3F1FF4F04DB2F
:1084280030EE400A03B05DF804FB684600F07EF8C1
:1084380000F0030001281AD002280FD000B3012051
:10844800DDED010A9DED000A00F082FDEAE7DFEDAF
:10845800110A00F0B3F903B05DF804FBDDED010A81
:108468009DED000A00F0AAF9B1EE400ADAE7DDED69
:10847800010A9DED000A00F06BFDB1EE400AD1E75C
:10848800DDED010A9DED000A00F098F9CAE700BF8A
:10849800D80F493F0000000000B510EE103A214AFD
:1084A80023F00043934283B01ADDB3F1FF4F04DB9E
:1084B80030EE400A03B05DF804FB684600F036F879
:1084C80000F0030001281DD0022811D008B3DDED0B
:1084D800010A9DED000A00F071F9B1EE400AE9E7E2
:1084E8000020DFED110A00F033FD03B05DF804FB56
:1084F8000120DDED010A9DED000A00F029FDB1EE35
:10850800400AD7E7DDED010A9DED000A00F056F9B3
:10851800D0E70120DDED010A9DED000A00F018FD0D
:10852800C8E700BFD80F493F0000000070B510EE43
:10853800103A944A23F00044944286B0054668DD18
:10854800914A944210EE106A1ADC002BDFED8F7A04
:108558008F4A24F00F0440F3DD80944270EE677A6E
:1085680066D09FED8C7A77EEC76A012077EEE67ABF
:10857800C5ED006A77EEC77AC5ED017A06B070BD21
:10858800854A944266DDB4F1FF4F49DAE215863A2E
:10859800A4EBC25307EE903ABDEEE77ADFED7F6AAF
:1085A800B8EEC77A77EEC77A8DED037A67EEA67ACA
:1085B800BDEEE77AB8EEC77A77EEC77A8DED047A22
:1085C80067EEA67AF5EE407AF1EE10FACDED057A6F
:1085D80040F0B380B5EE407AF1EE10FA0CBF0123FB
:1085E80002236F4901910221009103A8294600F056
:1085F80067F9002E12DA95ED007AD5ED017AB1EE21
:10860800477AF1EE677A404285ED007AC5ED017A46
:1086180004E0002285ED000A4260002006B070BD2B
:1086280070EE407A0020C5ED017AC5ED007AF5E7D5
:10863800DFED5C6A9FED5C7A77EEE67A012077EEF3
:10864800C76A77EEE67AC5ED006A77EEC77AC5EDB8
:10865800017AE3E700F0C4FCDFED546ADFED4B5A22
:10866800DFED4C7AB6EE007AA0EE267ABDEEC77A38
:10867800F8EEC76A17EE100AB1EE666A1F28A6EE72
:10868800250A66EEA77A1DDC494A411E24F0FF033D
:1086980052F82120934215D030EE677A85ED007AA2
:1086A80030EE470A002E30EE670A85ED010AB5DA8A
:1086B800B1EE477AB1EE400A85ED007A85ED010A00
:1086C8004042ABE730EE677AE41517EE103AC3F391
:1086D800C753E31A082BE1DDDFED327A9FED327ADA
:1086E800F0EE405AE6EE275A30EE650AA6EE270A63
:1086F800F0EE407AD6EE877A35EEE77A17EE103A42
:10870800C3F3C753E41A192C2CDC85ED007AB0EEBC
:10871800650AC5E7944270EE277A10D09FED1D7A5E
:1087280077EE876A4FF0FF3077EEE67AC5ED006A9C
:1087380077EE877AC5ED017A70E7032351E7DFED1D
:10874800196A9FED197A77EEA67A4FF0FF3077EE27
:10875800876A77EEE67AC5ED006A77EE877AC5ED27
:10876800017A5BE79FED137A9FED135AB0EE650A25
:10877800A6EE070A75EEC07AE6EE077AD6EE857A97
:108788008AE700BFD80F493FE3CB1640800FC93FA7
:10879800D00FC93F43443537800F49430000804319
:1087A8001C9700080044353708A3852E84F9223F1A
:1087B8009C96000800A3852E32318D2410EE103AC5
:1087C80023F00043B3F1485F2CDAFDEEC07A17EED0
:1087D800903A002B60D020EE007ADFED314A9FED11
:1087E800315ADFED315A9FED316ADFED317ADFED35
:1087F800316AA7EE245AE7EE055AA7EE256AE7EE96
:10880800067AE7EE276A66EE876A60EEC00AB6EE79
:10881800006AE7EE260AF7EE007AD7EE060A37EE88
:10882800E00A704720EE007ADFED1D4A9FED1D5AE1
:10883800DFED1D5A9FED1D6ADFED1D7ADFED1D6A24
:108848001D4AA7EE245A9342E7EE055AA7EE256A79
:10885800E7EE067AE7EE276A66EE876AD5DD174AFD
:10886800934214DC03F17F4307EE903AB7EE006AB7
:1088780036EE676A60EEC00AF6EE005AE7EE260AA0
:10888800D7EE257A77EEE07A36EE670A7047B6EECD
:10889800076AF5EE027AEDE7B7EE000A704700BF07
:1088A8004ED747ADF6740F317CF293B4010DD03733
:1088B800610BB6BAABAA2A3D9999993E0000483F88
:1088C8002DE9F04F2DED048BD9B003F1FF3A049355
:1088D800D31E48BF131DD44C669D0291DB1023EABA
:1088E800E373194654F8256006930133A2EBC303DA
:1088F8000193A1EB0A0316EB0A01814616D4194429
:108908009FEDCA7A679801311CAA002BA4BF50F8C2
:10891800234007EE904A03F10103ACBFF8EEE77A73
:10892800F0EE477A8B42E2EC017AEED1002EC0F2EB
:108938000783049B44AD9C00771C1CAB05EB8707A1
:10894800181909EB0401BAF1000FC0F27582DFEDC6
:10895800B77A4B460246F3EC016A32ED017A8B4254
:10896800E6EE877AF7D1E5EC017ABD4200F1040022
:10897800E9D106F18043013B9B0008AD1A1FAA18F4
:10898800B3460396DFEDAB8A9FEDA98A019E079255
:108998004C4405EB030844AF4FEA8B0358AA1A442A
:1089A800BBF1000F12ED140A18DD07A907EB8B02C3
:1089B80060EE287AB0EE407AFDEEE77A72ED016A51
:1089C800F8EEE77ABA42A7EEC87A37EEA60ABDEE05
:1089D800C77A17EE100A41F8040FE9D1304605931B
:1089E80000F04EFBB0EE409AB4EE000A29EE000A01
:1089F80000F0FEFAF2EE007AA0EE679A002E059BD0
:108A0800FDEEC99AF8EEE97A39EE679A40F3C98023
:108A18000BF1FF3EC6F1080255F82E1041FA02F09C
:108A280000FA02F2891A45F82E1019EE90EA8644E7
:108A3800C6F1070209EE90EA1141002951DD19EE4D
:108A4800902ABBF1000F02F1010209EE902A40F3CF
:108A580012822A68002A40F06982BBF1010F40F3B4
:108A68002982AE4601205EF8042F002A00F01E82FB
:108A780000F1010EC2F58072F34545F8202012DDA1
:108A880055F82E200230C2F1FF02834545F82E200A
:108A980009DD05EB8000EA180368C3F1FF0340F81D
:108AA800043B9042F8D1002E0DDD012E4FF001025B
:108AB80040F0E7810BF1FF3055F8203003F07F03D9
:108AC80045F82030E7E102290BD1F7EE007A37EEBE
:108AD800C99A3046B7EE000A00F0D2FA39EE409A49
:108AE8000221B5EE409AF1EE10FA70D1039B0BF11A
:108AF800FF3E73450EDC0BF18042013A05EB820222
:108B0800002052F80439424540EA0300F9D1002810
:108B180040F09480039B013B55F82330002B40F034
:108B2800D381079B4FF0010C53F804290CF1010C79
:108B3800002AF9D0DC440BF1010EE6452FDC069A39
:108B4800049B0EEB020103EB0B000CEB02031CAAC7
:108B580001F1804102EB8000679A013902EB810143
:108B680007EB8E0E02EB830B51F8043F07EE903AA9
:108B7800F8EEE77ABAF1000FE0EC017ADFED2B7A34
:108B880009DB4B460246F3EC016A32ED017AA34257
:108B9800E6EE877AF7D15945EEEC017AE4D1E3465F
:108BA800FAE605D10BF1FF3255F82210091244E715
:108BB800F6EE007AB4EEE79AF1EE10FA80F246810A
:108BC800B5EE409AF1EE10FA4FF000018ED0019CFC
:108BD800039EB0EE490A6042884600F051FA9FEDC4
:108BE800147AB4EEC70AF1EE10FAC0F28581DFED0F
:108BF800117A60EE277A2346FDEEE77A0833F8EE1D
:108C0800E77A0193A7EEC70A0BF10103FDEEE77AB5
:108C1800BDEEC00A10EE102A45F82B2017EE902A58
:108C280045F823201FE000BF609A000800000000FC
:108C3800000080430000803B0000C93F884601993E
:108C480055F82E20039E0839734601915AB90EF142
:108C58008042013A05EB820252F80409013B0839C7
:108C68000028F9D0019101980393B7EE000A00F0AB
:108C780007FA039B002BC0F24A819F0044AAD0192F
:108C880007F1040E1FED157A05EB0E02011D72EDBA
:108C9800017AF8EEE77AAA4267EE807A20EE070AB0
:108CA80061ED017AF3D11FED1C6A05460DF5867C4E
:108CB8000024002EC0F2DC80A348DFEDA47A294608
:108CC800B0EE467A002203E0A24208DCB0EC017A5A
:108CD800F1EC016A01329642E7EE267AF4DA043DB5
:108CE80058AA02EB8402654542ED287A04F1010492
:108CF800DFD1669A032A5AD8DFE802F08C62620252
:108D0800002B40F3018158AA3A4430A912ED287A81
:108D18003A1D0A4431A8394451ED017A77EE876A41
:108D280077EEE67A77EE877AB0EE667A62ED017AC8
:108D3800824261ED016AEFD1012B40F3E58058AB27
:108D48003B4430AA13ED287A3B1D32A917441A4434
:108D580057ED017A77EE876A77EEE67A77EE877ACB
:108D6800B0EE667A62ED017A914267ED016AEFD161
:108D780030A9DFED767A0B4433ED017A9A4277EE2B
:108D8800877AF9D14346002B00F0AE80DDED306ADA
:108D98009DED317A029AF1EE677AF1EE666AB1EEEC
:108DA800477AC2ED027AC2ED006A82ED017A19EEC5
:108DB800903A03F0070059B0BDEC048BBDE8F08F82
:108DC8003A1D30A9DFED617A0A4432ED017A8A4210
:108DD80077EE877AF9D14246002A78D0DDED306AFD
:108DE800029AB1EE677A002B76EEE77A82ED007A86
:108DF8000ADD31A90122B1EC017A0132934277EE02
:108E0800877AF8DA43460BB1F1EE677A029BC3ED35
:108E1800017ACCE730ABDFED4D7A9E443EED017A26
:108E2800734577EE877AF9D143460BB1F1EE677A4D
:108E3800029BC3ED007ABAE7DFED447AE5EC017AEC
:108E4800BD4200F104007FF47EAD92E519EE902A50
:108E5800BBF1000F02F1010209EE902AC8BF0221FE
:108E68003FF7F7ADF7EE007A37EEC99A022138E6F8
:108E7800DFED367A33E7002E1EDD0022012E3FF4A7
:108E880019AE022E07D10BF1FF3055F8203003F050
:108E98003F0345F8203002297FF423AEF7EE007A2D
:108EA80037EEC99A002A3FF41CAE12E6013083451A
:108EB8007FF4D9AD002EE1DC02297FF412AEF7EE83
:108EC800007A37EEC99A0CE64FF0010C32E69DEDB8
:108ED800307A029A002BC2ED007A77EE677A88DC46
:108EE800029BC3ED017A62E70298309A319BC0ED8C
:108EF800027A026043605AE7BDEEC00A5B4610EE94
:108F0800102A45F82B20AEE6DFED107A3AE7669A8C
:108F1800032A3FF64CAF01A151F822F0438F000815
:108F28003D8F00083D8F0008118F00084FF0010E9B
:108F380000209FE5DFED057A4DE7DFED047A73E762
:108F4800049B9C0015E500BF389A0008000000004B
:108F580010EE103A23F00043B3F1485F04DAFDEE57
:108F6800C07A17EE903A23B360EE007A9FED155A57
:108F7800DFED155A9FED156ADFED156A9FED157A3D
:108F8800E7EE855A20EE275AA7EEA56AE7EE866A2D
:108F9800A7EEA67A70B127EE457AF6EE006AA0EE43
:108FA800A67ADFED0D6AD7EE870AE5EE260A30EEDF
:108FB800600A7047DFED096AE7EE876AA5EE260AC0
:108FC800704700BFD3C92E2F342FD7B21BEF3836C6
:108FD800010D50B98988083CABAA2A3EABAA2ABE23
:108FE80010EE103A23F0004300EE103A704700BF2D
:108FF80010EE102A22F00041CB0D7F3B162B17DC18
:10900800002B10EE100A19DB1A4919410A4222D026
:10901800DFED197A70EE277AF5EEC07AF1EE10FAE4
:1090280019DD002A18DB20EA010300EE103A704728
:10903800B1F1FF4F0FD330EE000A7047DFED0E7A23
:1090480070EE277AF5EEC07AF1EE10FA03DD002A09
:1090580008DB9FED0A0A70474FF4000242FA03F357
:109068001844E0E70029FFEE007A18BFB0EE670A5F
:10907800704700BFFFFF7F00CAF24971000000007F
:1090880008B510EE103A33F000422DED028B11D0E6
:10909800B2F1FF4F11D2B2F5000F13D3D20D024433
:1090A800FE2A2EDC002A1ADD23F0FF4343EAC253CE
:1090B80000EE103ABDEC028B08BDBDEC028B30EE21
:1090C800000A08BD1D4BDFED1E7A984220EE270AE4
:1090D80022DB10EE103AC3F3C752193ADFE712F158
:1090E800160F1EDA4CF2503398420ADC9FED158AAF
:1090F800F0EE400AB0EE480A00F02AF820EE080A1E
:10910800D8E79FED118AF0EE400AB0EE480A00F069
:109118001FF820EE080ACDE7DFED0A0A20EE200A44
:10912800C8E7193223F0FF4343EAC253DFED077A59
:1091380000EE103A20EE270ABCE700BFB03CFFFF64
:109148000000004C6042A20DCAF2497100000033D1
:1091580010EE103A10EE902A23F0004302F000427D
:10916800134300EE103A704710B5431E0A4491426B
:1091780000D110BD11F8014B03F8014FF7E7884201
:1091880010B501EB020303D8421E99420CD110BD61
:109198009842F9D28118D21AD34200D110BD13F8DF
:1091A800014D01F8014DF7E711F8014B02F8014FA5
:1091B800EBE702440346934200D1704703F8011BD2
:1091C800F9E700000000000000380140000000003E
:1091D800000000001A273500192634004E072550D4
:1091E800500000000200000000480040000000009D
:1091F800000000002B3B00002A3A000072072740BD
:109208005000000000000000005400401F26281EE7
:109218002729750000000000000000000000000081
:10922800000000000000000080250000004B000046
:109238000096000000E1000000C201000084030065
:1092480090D00300801A06000008070020A107003C
:1092580000100E0040420F0060E3160080841E00DC
:1092680070B02500011D0008651C0008B11B00082E
:1092780000020000000000000004000000000000E0
:10928800000800000000000000100000741C00200E
:10929800741D0020FFFF0000000000006E0A01009E
:1092A800002C01404B1B000000000040601C000027
:1092B80000040040611D000000080040621E00001C
:1092C8000010004064000000001400406500000029
:1092D800003401404D2E00000040014050180000AD
:1092E800004401405119000000480140521A000092
:1092F8003132333435360000B10F0008251000082C
:10930800C91000084113000819100008E10F0008EF
:10931800C50F0008B90F0008B50F00089110000824
:10932800A90F0008393A0008813900087539000882
:10933800B13A0008953900088D39000891390008BC
:10934800593A000879390008313A00081400020037
:109358000010203031310000FFFFFFFFFFFF040045
:1093680000001300012F0008012F0008ED65000818
:10937800012F0008012F0008012F0008012F000805
:1093880039660008012F0008012F0008012F000886
:10939800012F0008012F0008012F0008991D00085F
:1093A800B11E00087D1E0008291E00086943000838
:1093B800651E0008AB420008000000000000000025
:1093C8000000000000040040200804010200000022
:1093D8001C0002400100000000040040210C0401B0
:1093E800020000003000024002000000004401407A
:1093F80024000401010000006C0002400500000088
:1094080000480140250004010A00000080000240D5
:1094180006000000002C0140180020000600000093
:109428001C000240010000000000000000000000D5
:109438000000000000000000000000000000000024
:109448000000000000000000000000000000000014
:109458000000000000000000000000000000000004
:1094680000000000000000000000000000000000F4
:1094780000000000000000000000000000000000E4
:1094880000000000000000000000000000000000D4
:1094980000000000000000000000000000000000C4
:1094A80000000000000000000000000000000000B4
:1094B80000000000010694111027020994111027DA
:1094C8000301E4578813000000090408030906078C
:1094D80001060907080206000100123456789ABCF2
:1094E80000000000100111021203130414011502F8
:1094F80016031704200C2101220C2C032D052E0421
:109508002F0530063107320833093405350B000CB6
:10951800000D000700080009000A000B000D0006F6
:109528000002000E000F0010000300010002000AF4
:109538006405000012010002020000408304405745
:1095480000020102030100003203530054004D00E1
:109558003300320020005600690072007400750064
:1095680061006C00200043004F004D0020005000B7
:109578006F007200740020002000000026035300D2
:1095880054004D006900630072006F0065006C00B4
:1095980065006300740072006F006E00690063006C
:1095A80073000000040309040401000009024300D9
:1095B800020100C032090400000102020100052472
:1095C80000100105240100010424020205240600FC
:1095D80001070582030800FF09040100020A0000D0
:1095E8000007050302400000070581024000000053
:1095F8004254464C000000004F637420203920324A
:109608003031370031303A34333A32340000000018
:10961800356262346566323464000000574149544B
:10962800494E4720464F522046430000332E322EE3
:1096380030000000562573004F53440053595354CB
:10964800454D000053455249414C00004241545495
:109658004552595F564F4C54414745004241545476
:109668004552595F43555252454E54004241545455
:109678004552595F414C4552545300005452414E93
:1096880053504F4E444552004F53445F534C41563C
:1096980045000000000FC93F000F494000CB96402D
:1096A800000FC9400053FB4000CB164100ED2F418D
:1096B800000F49410031624100537B41003A8A4121
:1096C80000CB9641005CA34100EDAF41007EBC4158
:1096D800000FC94100A0D5410031E24100C2EE416E
:1096E8000053FB4100F20342003A0A420083104251
:1096F80000CB164200141D42005C234200A52942FB
:1097080000ED2F4200363642007E3C4200C74242FE
:10971800000F4942A2000000F90000008300000089
:109728006E0000004E00000044000000150000001C
:1097380029000000FC00000027000000570000007E
:10974800D1000000F500000034000000DD0000003A
:10975800C0000000DB00000062000000950000006F
:10976800990000003C000000430000009000000049
:1097780041000000FE0000005100000063000000EE
:10978800AB000000DE000000BB000000C5000000C8
:1097980061000000B7000000240000006E00000017
:1097A8003A000000420000004D000000D200000016
:1097B800E000000006000000490000002E00000044
:1097C800EA00000009000000D1000000920000003B
:1097D8001C000000FE0000001D000000EB0000005F
:1097E8001C000000B100000029000000A7000000D4
:1097F8003E000000E8000000820000003500000084
:10980800F50000002E000000BB000000440000002E
:1098180084000000E90000009C00000070000000C7
:1098280026000000B40000005F0000007E00000079
:10983800410000003900000091000000D60000003F
:1098480039000000830000005300000039000000C8
:10985800F40000009C000000840000005F0000008D
:109868008B000000BD000000F90000002800000087
:109878003B0000001F000000F800000097000000F7
:10988800FF000000DE000000050000009800000056
:109898000F000000EF0000002F0000001100000082
:1098A8008B0000005A0000000A0000006D00000054
:1098B8001F0000006D000000360000007E00000060
:1098C800CF00000027000000CB00000009000000C6
:1098D800B70000004F000000460000003F000000F5
:1098E800660000009E0000005F000000EA00000023
:1098F8002D0000007500000027000000BA000000DD
:10990800C7000000EB000000E5000000F1000000C7
:109918007B0000003D000000070000003900000047
:10992800F70000008A0000005200000092000000CA
:10993800EA0000006B000000FB0000005F00000070
:10994800B10000001F0000008D0000005D00000055
:10995800080000005600000003000000300000006E
:1099680046000000FC0000007B0000006B000000C7
:10997800AB000000F0000000CF000000BC000000B9
:10998800200000009A000000F400000036000000EB
:109998001D000000A9000000E30000009100000085
:1099A800610000005E000000E60000001B000000EF
:1099B8000800000065000000990000008500000014
:1099C8005F00000014000000A00000006800000014
:1099D800400000008D000000FF000000D8000000DB
:1099E800800000004D000000730000002700000008
:1099F800310000000600000006000000150000000D
:109A080056000000CA00000073000000A800000013
:109A1800C900000060000000E20000007B000000B8
:109A2800C00000008C0000006B0000000000C93F6F
:109A38000000F0390000DA370000A2330000842E5D
:109A48000000502B0000C2270000D0220000C41FD5
:109A58000000C61B000044170400000007000000B7
:049A680009000000F1
:109A6C0013000400080C0020100C00200000000063
:109A7C00C09B000812100800000C0020140C0020E1
:109A8C0000000000C49B00080201030088120020A3
:109A9C0084120020000000003910000801020500AB
:109AAC00380E00208C120020000000002910000845
:109ABC00FE01080098130020901300200000000005
:109ACC00A11B00080D001C00C81300201816002054
:109ADC00000000001D5A000802020300BC13002005
:109AEC00341600200000000000000000F901040002
:109AFC00F8160020F4160020000000009D4200081B
:109B0C00FD011E001C170020FC16002000000000A8
:109B1C008542000811000C0090170020881A0020C4
:109B2C0000000000D559000800010400D41A0020E0
:109B3C00B41B002000000000CC9B00080B20100080
:109B4C00A81A0020B81B002000000000D09B0008C1
:109B5C0006020800D01B0020C81B002000000000DB
:109B6C00D35F000808020900E41B0020D81B00206A
:109B7C0000000000A95F00080C020100F81B002087
:109B8C00F41B002000000000E09B00082F001100D7
:109B9C00101C0020FC1B002000000000E29B0008B1
:109BAC00F70106002C1C0020241C002000000000E3
:049BBC00F49B00080E
:109BC000002020000001534F4633000090010000A8
:109BD0002B21231E64010100000001000A0129005D
:109BE0000100000000000000000000000000000074
:0A9BF000000000000000010000006A
:109BFA00E0010800FFFF000000000000010203046A
:109C0A000102030406070809010002000400060015
:109C1A0008000A000C00100020004000800000012B
:109C2A0000000000000000003568000845660008D2
:109C3A00B5650008B1650008516500082D65000882
:109C4A009D64000809650008E5640008AD64000821
:109C5A000000000040000000012F0008D565000840
:109C6A00012F0008012F0008012F0008012F00080A
:109C7A00012F0008012F0008C965000800C2010071
:109C8A000000080000000240080002400000000036
:109C9A00000B0000010000000000000000000000AE
:109CAA00000002401C00024000000000040C0000FA
:109CBA000100000000000000000000000000024057
:109CCA003000024000000000080D00000100000002
:109CDA0000000000000000000000024044000240B2
:109CEA00000000000C0E000001000000000000004F
:109CFA00000000000000024058000240000000007E
:109D0A00100F000001000000000000000000000029
:109D1A00000002406C000240000000001410000025
:109D2A0001000000000000000000000000000240E6
:109D3A00800002400000000018110000010000002D
:109D4A000000000000000000000402400804024075
:109D5A0000000000003800000200000000000000BF
:109D6A0000000000000402401C0402400000000041
:109D7A00043900000200000000000000000000009A
:109D8A00000402403004024000000000083A0000CB
:109D9A000200000000000000000000000004024071
:109DAA0044040240000000000C3B000002000000D6
:109DBA0000000000000000000004024058040240B5
:109DCA0000000000103C000002000000000000003B
:109DDA000000000044960008000000000000000097
:109DEA00D1580008A086010004000000000000000D
:109DFA000000000000000000000000000000000059
:109E0A000000000000000000000000000000000048
:109E1A000000000000000000000000000000000038
:109E2A000000000000000000000000000000000028
:109E3A000000000000000000000000000000000018
:109E4A000000000000000000000000000000000008
:109E5A0000000000000000000000000000000000F8
:109E6A0000000000000000000000000000000000E8
:109E7A0000000000000000000000000000000000D8
:109E8A0000000000000000000000000000000000C8
:109E9A0000000000000000000000000000000000B8
:109EAA0000000000000000000000000000000000A8
:109EBA000000000000000000000000000000000098
:109ECA000000000000000000000000000000000088
:109EDA0000000000000000004C960008000000008E
:109EEA00691B00088901000810270000060000000D
:109EFA000000000000000000000000000000000058
:109F0A000000000000000000000000000000000047
:109F1A000000000000000000000000000000000037
:109F2A000000000000000000000000000000000027
:109F3A000000000000000000000000000000000017
:109F4A00549600080000000000000000F9570008BD
:109F5A00204E000003000000000000000000000086
:109F6A0000000000000000000000000000000000E7
:109F7A0000000000649600080000000000000000D5
:109F8A0005570008204E00000300000000000000F2
:109F9A0000000000000000000000000000000000B7
:109FAA000000000000000000749600080000000095
:109FBA0000000000296D0008400D030003000000A6
:109FCA000000000000000000000000000000000087
:109FDA000000000000000000000000008496000855
:109FEA00000000000000000001590008A00F000056
:109FFA000100000000000000000000000000000056
:10A00A000000000000000000000000000000000046
:10A01A009096000800000000491000087D0F000813
:10A02A001A410000050000000000000000000000C6
:10A03A000000000000000000000000000000000016
:10A04A0000000000AC950008040000008495000898
:10A05A002600000050950008320000008404002009
:10A06A001A000000B4950008430000003C9500085F
:10A07A00120000001A03530054004D00330032004E
:10A08A0000000000000000000000000000000000C6
:10A09A0001000000000000000000000001020304AB
:08A0AA0006070809010000008F
:0400000508000000EF
:00000001FF
